:030000000269BFD3
:1069BF00758E1190000078FF79FFE4F0A3D9FBD812
:0D69CF00F778FFE4F6D8FD75817F026A17A6
:106DB2004401EA40490FDB4401E640C90FDB4401CC
:056DC200E23C8EFA35F1
:064A3E009001CA122028BD
:104A44009001CEE0FCA3E0FDA3E0FEA3E0FFEF2491
:104A540069FFEE3474FEED34FFFDEC34FFFCEC1220
:104A64001B927BDF7A927986783D12196E9001D27F
:104A74001220287B007A0079C078419001D2E0FCB2
:104A8400A3E0FDA3E0FEA3E0FF121A771263117BFB
:104A9400007A0079C0784112196EC004C005C006BE
:104AA400C0077F977E7E7DD57C409001D2E0F8A33D
:104AB400E0F9A3E0FAA3E0FB12187DD003D002D002
:104AC40001D000121879C004C005C006C0077F9247
:104AD4007E867DC07C419001CAE0F8A3E0F9A3E0A2
:104AE400FAA3E0FB12196EA804A905AA06AB07D025
:104AF40007D006D005D00412187D9001DA122028C0
:104B04009001CEE0FCA3E0FDA3E0FEA3E0FFEF24D0
:104B140069FFEE3474FEED34FFFDEC34FFFCEC125F
:104B24001B929001CAE0F8A3E0F9A3E0FAA3E0FB2A
:104B340012187D7B307AE67958783D12196EA804F4
:104B4400A905AA06AB077F817E0E7DBA7C431218A5
:104B5400799001E2E0F8A3E0F9A3E0FAA3E0FB1204
:104B6400196E9001D61220289001E6E0FCA3E0FD26
:104B7400A3E0FEA3E0FF9001D6E0F8A3E0F9A3E0F0
:104B8400FAA3E0FB121B14602940279001D6E0FC35
:104B9400A3E0FDA3E0FEA3E0FF9001E6E0F8A3E0BC
:104BA400F9A3E0FAA3E0FB1218799001D6122028A9
:104BB40080B69001E6E0FCA3E0FDA3E0FEA3E0FFE5
:104BC400121B819001D6E0F8A3E0F9A3E0FAA3E078
:104BD400FB121B1450279001D6E0FCA3E0FDA3E0D8
:104BE400FEA3E0FF9001E6E0F8A3E0F9A3E0FAA356
:104BF400E0FB12187D9001D612202880B57F007E3C
:104C0400007D007C009001D6E0F8A3E0F9A3E0FA6F
:104C1400A3E0FB121B14604840469001EAE0FCA3A9
:104C2400E0FDA3E0FEA3E0FF9001D6E0F8A3E0F9E5
:104C3400A3E0FAA3E0FB121B1450259001D6E0FC7C
:104C4400A3E0FDA3E0FEA3E0FF9001E6E0F8A3E00B
:104C5400F9A3E0FAA3E0FB1218799001D6122028F8
:104C64007F007E007D007C009001D6E0F8A3E0F98F
:104C7400A3E0FAA3E0FB121B14504B9001EAE0FC02
:104C8400A3E0FDA3E0FEA3E0FF121B819001D6E0A8
:104C9400F8A3E0F9A3E0FAA3E0FB121B1460274099
:104CA400259001D6E0FCA3E0FDA3E0FEA3E0FF9085
:104CB40001E6E0F8A3E0F9A3E0FAA3E0FB12187D13
:104CC4009001D61220289001D6E0FCA3E0FDA3E0D9
:104CD400FEA3E0FF125A617B247A0B79987839128B
:104CE400196E9001DAE0F8A3E0F9A3E0FAA3E0FB7F
:104CF40012187D9001DE1220287B007A0079C0789A
:104D0400419001DEE0FCA3E0FDA3E0FEA3E0FF127E
:104D14001A771263117B007A0079C0784112196EF8
:104D2400A804A905AA06AB079001DEE0FCA3E0FDF8
:094D3400A3E0FEA3E0FF121879D0
:014D3D002253
:106E3F009001F51220289001F5E0FCA3E0FDA3E0FE
:106E4F00FEA3E0FF126311A804A905AA06AB0790E1
:106E5F0001F5E0FCA3E0FDA3E0FEA3E0FF1218792B
:106E6F009001E6E0F8A3E0F9A3E0FAA3E0FB121922
:026E7F006E2281
:060D470090015A12202861
:100D4D0090015AE0FCA3E0FDA3E0FEA3E0FFEF2439
:100D5D0013FFEE342DFEED34FFFDEC34FFFCEC12F1
:100D6D001B9290015EE0F8A3E0F9A3E0FAA3E0FB8B
:100D7D0012187D9001621220287F8D7EA67D147C35
:100D8D003D900162E0F8A3E0F9A3E0FAA3E0FB12C5
:100D9D00196E7B807AF279BF783E12187D126E3F04
:100DAD009001661220287F477E857D167C3D90013F
:100DBD0062E0F8A3E0F9A3E0FAA3E0FB12196E7B61
:100DCD00937AA77984783E12187D126E3F90016A4E
:100DDD001220287F217EB47D0A7C3D900162E0F8CF
:100DED00A3E0F9A3E0FAA3E0FB12196E7BFF7ACD25
:100DFD007953783F12187D126E3F90016E122028A4
:100E0D007F4D7E6C7D337C3B900162E0F8A3E0F971
:100E1D00A3E0FAA3E0FB12196E7B817A3D797E780F
:100E2D003F12187D126E3F9001721220287F007EB6
:100E3D00007D007C4090016EE0F8A3E0F9A3E0FA9C
:100E4D00A3E0FB12196EA804A905AA06AB07900131
:100E5D0066E0FCA3E0FDA3E0FEA3E0FF121879120B
:100E6D005A4B7BF37A767914783F12196EC004C011
:100E7D0005C006C007900166E0FCA3E0FDA3E0FEFF
:100E8D00A3E0FF125A4B7BE87AC1795178401219D1
:100E9D006EA804A905AA06AB077FB17E737D717C90
:100EAD0042121879D003D002D001D000121879C0A7
:100EBD0004C005C006C0077F007E007D007C409009
:100ECD00016EE0F8A3E0F9A3E0FAA3E0FB12196EBE
:100EDD00125A4B7B0C7A5979ED783E12196EA80493
:100EED00A905AA06AB07D007D006D005D004121865
:100EFD00799001761220287F007E007D007C409045
:100F0D00016EE0F8A3E0F9A3E0FAA3E0FB12196E7D
:100F1D00C004C005C006C0077F007E007D007C4078
:100F2D00900166E0F8A3E0F9A3E0FAA3E0FB121943
:100F3D006ED003D002D001D000121879125A4B7B1B
:100F4D00767A4F791E783D12196EC004C005C00621
:100F5D00C0077F007E007D007C40900166E0F8A315
:100F6D00E0F9A3E0FAA3E0FB12196E125A4B7B9C39
:100F7D007A5A79B6783D12196EA804A905AA06AB5E
:100F8D0007900176E0FCA3E0FDA3E0FEA3E0FF12D5
:100F9D001879A804A905AA06AB07D007D006D00575
:100FAD00D00412187DC004C005C006C0077F007EA6
:100FBD00007D007C4090016EE0F8A3E0F9A3E0FA1B
:100FCD00A3E0FB12196E900172E0F8A3E0F9A3E023
:100FDD00FAA3E0FB121879125A4B7B687A967904C2
:100FED00783D12196EA804A905AA06AB07D007D043
:100FFD0006D005D0041218799001761220287F00B2
:10100D007E007D007C4090016EE0F8A3E0F9A3E046
:10101D00FAA3E0FB12196EA804A905AA06AB079066
:10102D000166E0FCA3E0FDA3E0FEA3E0FF1218794A
:10103D00900172E0F8A3E0F9A3E0FAA3E0FB121827
:10104D007D125A4B7BD87A2A79C1783C12196EC021
:10105D0004C005C006C0077F007E007D007C409067
:10106D00016EE0F8A3E0F9A3E0FAA3E0FB12196E1C
:10107D00A804A905AA06AB07900166E0FCA3E0FD54
:10108D00A3E0FEA3E0FF121879125A4B7B727A335C
:10109D0079DC783C12196EA804A905AA06AB079055
:1010AD000176E0FCA3E0FDA3E0FEA3E0FF121879BA
:1010BD00D003D002D001D000121879C004C005C0F1
:1010CD0006C007900172E0F8A3E0F9A3E0FAA3E0EF
:1010DD00FB900166E0FCA3E0FDA3E0FEA3E0FF12A0
:1010ED001879125A4B7B307A4C79A6783C12196ECE
:1010FD00A804A905AA06AB07D007D006D005D004D1
:10110D0012187990017612202890016EE0FCA3E070
:10111D00FDA3E0FEA3E0FF125A4B7B0B7AD2798C34
:10112D00783C12196E900176E0F8A3E0F9A3E0FA8D
:10113D00A3E0FB12187DC004C005C006C0079001D6
:10114D0072E0FCA3E0FDA3E0FEA3E0FF900166E0EA
:10115D00F8A3E0F9A3E0FAA3E0FB12187D125A4BB5
:10116D007B697AE37988783C12196EA804A905AADF
:10117D0006AB07D007D006D005D00412187D90011C
:10118D00761220287F007E007D007C4090016AE071
:10119D00F8A3E0F9A3E0FAA3E0FB12196EA804A9E5
:1011AD0005AA06AB07900166E0FCA3E0FDA3E0FEF7
:1011BD00A3E0FF121879125A4B7BF97A4E794C78CD
:1011CD003C12196EC004C005C006C007900172E044
:1011DD00FCA3E0FDA3E0FEA3E0FF125A4B7BCD7A0A
:1011ED00AF79E6783B12196EA804A905AA06AB07DC
:1011FD00D007D006D005D00412187DC004C005C09C
:10120D0006C0077F007E007D007C4090016EE0F8F7
:10121D00A3E0F9A3E0FAA3E0FB12196E900172E0CE
:10122D00F8A3E0F9A3E0FAA3E0FB12187D125A4BE4
:10123D007BBC7A5779AD783B12196EA804A905AA23
:10124D0006AB07D007D006D005D00412187DC00418
:10125D00C005C006C0077F007E007D807C409001E8
:10126D006EE0F8A3E0F9A3E0FAA3E0FB12196EA873
:10127D0004A905AA06AB07900166E0FCA3E0FDA357
:10128D00E0FEA3E0FF121879125A4B7B4E7AB47927
:10129D00AB783B12196EA804A905AA06AB07D007B7
:1012AD00D006D005D00412187990017A1220287F2B
:1012BD00007E007D007C4090016EE0F8A3E0F9A374
:1012CD00E0FAA3E0FB12196EA804A905AA06AB0764
:1012DD00900166E0FCA3E0FDA3E0FEA3E0FF121881
:1012ED0079900172E0F8A3E0F9A3E0FAA3E0FB1214
:1012FD001879125A4B7BA97A6A7982783B12196E4A
:10130D0090017AE0F8A3E0F9A3E0FAA3E0FB12184C
:10131D007DC004C005C006C0077F007E007D407CF7
:10132D0040900166E0F8A3E0F9A3E0FAA3E0FB1218
:10133D00196E125A4B7B9C7ADC796F783B12196EC1
:10134D00A804A905AA06AB07D007D006D005D0047E
:10135D00121879C004C005C006C0077F007E007D4D
:10136D00807C4090016EE0F8A3E0F9A3E0FAA3E0E1
:10137D00FB12196EC004C005C006C0077F007E00B9
:10138D007D007C40900166E0F8A3E0F9A3E0FAA3AC
:10139D00E0FB12196ED003D002D001D000121879E3
:1013AD00125A4B7BCA7A547941783B12196EA804B4
:1013BD00A905AA06AB07D007D006D005D004121890
:1013CD007990017A1220287F007E007D007C40906C
:1013DD00016EE0F8A3E0F9A3E0FAA3E0FB12196EA9
:1013ED00C004C005C006C0077F007E007D407C4064
:1013FD00900166E0F8A3E0F9A3E0FAA3E0FB12196F
:10140D006ED003D002D001D000121879125A4B7B46
:10141D00457A2F7923783B12196EC004C005C0069A
:10142D00C007900172E0FCA3E0FDA3E0FEA3E0FF86
:10143D0090016EE0F8A3E0F9A3E0FAA3E0FB121827
:10144D007D125A4B7B147A5C792C783B12196EA85D
:10145D0004A905AA06AB0790017AE0FCA3E0FDA361
:10146D00E0FEA3E0FF121879A804A905AA06AB07B0
:10147D00D007D006D005D00412187DC004C005C019
:10148D0006C0077F007E007D007C4090016EE0F875
:10149D00A3E0F9A3E0FAA3E0FB12196E900166E058
:1014AD00F8A3E0F9A3E0FAA3E0FB12187D90017216
:1014BD00E0F8A3E0F9A3E0FAA3E0FB121879125AC1
:1014CD004B7BA67AD57910783B12196EA804A90525
:1014DD00AA06AB07D007D006D005D004121879C0E4
:1014ED0004C005C006C0077F007E007D007C4090D3
:1014FD00016EE0F8A3E0F9A3E0FAA3E0FB12196E88
:10150D00C004C005C006C0077F007E007D007C4082
:10151D0090016AE0F8A3E0F9A3E0FAA3E0FB121949
:10152D006ED003D002D001D000121879125A4B7B25
:10153D00B37A7B79F2783A12196EA804A905AA0636
:10154D00AB07D007D006D005D00412187D90017AD4
:10155D001220287F007E007D007C4090016AE0F81B
:10156D00A3E0F9A3E0FAA3E0FB12196E900166E087
:10157D00F8A3E0F9A3E0FAA3E0FB12187DC004C0C4
:10158D0005C006C0077F007E007D007C4090016E87
:10159D00E0F8A3E0F9A3E0FAA3E0FB12196EA804AA
:1015AD00A905AA06AB07D007D006D005D00412189E
:1015BD0079125A4B7B047AAD79C0783A12196EC004
:1015CD0004C005C006C0077F007E007D007C4090F2
:1015DD000172E0F8A3E0F9A3E0FAA3E0FB12196EA3
:1015ED00C004C005C006C0077F007E007D007C40A2
:1015FD0090016EE0F8A3E0F9A3E0FAA3E0FB121965
:10160D006ED003D002D001D000121879125A4B7B44
:10161D00A37A0679D378BA12196EA804A905AA0679
:10162D00AB07D007D006D005D00412187DC004C07A
:10163D0005C006C0077F007E007D807C4090016E56
:10164D00E0F8A3E0F9A3E0FAA3E0FB12196E125A39
:10165D004B7B4B7A1F79BA783A12196EA804A905FB
:10166D00AA06AB07D007D006D005D004121879C052
:10167D0004C005C006C0077F007E007D007C409041
:10168D00016EE0F8A3E0F9A3E0FAA3E0FB12196EF6
:10169D00C004C005C006C0077F007E007D007C40F1
:1016AD00900166E0F8A3E0F9A3E0FAA3E0FB1219BC
:1016BD006ED003D002D001D000121879900172E0E3
:1016CD00F8A3E0F9A3E0FAA3E0FB12187D125A4B40
:1016DD007BA97A3079B6783A12196EA804A905AAB1
:1016ED0006AB07D007D006D005D00412187D9001A7
:1016FD007E1220287F007E007D807C4090016EE070
:10170D00F8A3E0F9A3E0FAA3E0FB12196EA804A96F
:10171D0005AA06AB07900166E0FCA3E0FDA3E0FE81
:10172D00A3E0FF121879900172E0F8A3E0F9A3E0AD
:10173D00FAA3E0FB12187D125A4B7B3B7AAA799AD9
:10174D00783A12196EA804A905AA06AB0790017E76
:10175D00E0FCA3E0FDA3E0FEA3E0FF121879C004B6
:10176D00C005C006C0077F007E007D007C40900153
:10177D006EE0F8A3E0F9A3E0FAA3E0FB12196EC046
:10178D0004C005C006C0077F007E007D007C409030
:10179D000166E0F8A3E0F9A3E0FAA3E0FB12196EED
:1017AD00A804A905AA06AB07D007D006D005D0041A
:1017BD0012187D125A4B7B247A0B7998783A1219AC
:1017CD006EA804A905AA06AB07D007D006D005D090
:1017DD0004121879C004C005C006C0077F007E0042
:1017ED007D007C40900166E0F8A3E0F9A3E0FAA348
:1017FD00E0FB12196E900172E0F8A3E0F9A3E0FA94
:10180D00A3E0FB121879125A4B7BE07A2D79907870
:10181D003A12196EA804A905AA06AB07D007D0067F
:10182D00D005D00412187990017E12202890017AEB
:10183D00E0FCA3E0FDA3E0FEA3E0FF900176E0F85D
:10184D00A3E0F9A3E0FAA3E0FB12187D90017EE07E
:10185D00F8A3E0F9A3E0FAA3E0FB12187D7B487A28
:08186D005179C7784512196E8C
:011875002250
:0B2B9400900120EBF0A3EAF0A3E9F0B1
:102B9F00900126E0FCA3E0FDA3E0FEA3E0FFEC1212
:102BAF001B927B007A81798878C612187D90012A52
:102BBF00E0F8A3E0F9A3E0FAA3E0FB12187D90017F
:102BCF002E1220287F0A7EEB7D157C3D90012EE092
:102BDF00F8A3E0F9A3E0FAA3E0FB12196E7B7F7A6A
:102BEF004F7940783F12187D126E3F9001321220BC
:102BFF00287F8C7EA67D147C3D90012EE0F8A3E00B
:102C0F00F9A3E0FAA3E0FB12196E7B367A907952A2
:102C1F00783F12187D126E3F9001361220287F4D9B
:102C2F007E6C7D337C3B90012EE0F8A3E0F9A3E0AE
:102C3F00FAA3E0FB12196E7B857AEA797E783F1250
:102C4F00187D126E3F90013A1220287F217EB47DAD
:102C5F000A7C3D90012EE0F8A3E0F9A3E0FAA3E08F
:102C6F00FB12196E7BD37A697979783F12187D122E
:102C7F006E3F90013E1220287F477E857D167C3D5A
:102C8F0090012EE0F8A3E0F9A3E0FAA3E0FB1219FC
:102C9F006E7B9F7A027900783D12187D126E3F90FD
:102CAF0001421220287F007E007D007C4090013E73
:102CBF00E0F8A3E0F9A3E0FAA3E0FB12196E125AB1
:102CCF00617BB07A727928783F12196EC004C00503
:102CDF00C006C007900136E0FCA3E0FDA3E0FEA311
:102CEF00E0FF125A617B7D7A3F79C9784012196EE5
:102CFF00A804A905AA06AB07D007D006D005D004B3
:102D0F0012187DC004C005C006C0077F007E007D7D
:102D1F00007C4090013EE0F8A3E0F9A3E0FAA3E0C5
:102D2F00FB12196EA804A905AA06AB07900136E09D
:102D3F00FCA3E0FDA3E0FEA3E0FF121879125A6195
:102D4F007B6F7A1279A3783F12196EA804A905AA8E
:102D5F0006AB07D007D006D005D004121879C004EF
:102D6F00C005C006C00790013AE0FCA3E0FDA3E058
:102D7F00FEA3E0FF125A617BC97A76793E783E1244
:102D8F00196EA804A905AA06AB07D007D006D0056F
:102D9F00D0041218799001E2E0F8A3E0F9A3E0FA69
:102DAF00A3E0FB12196E900132E0F8A3E0F9A3E063
:102DBF00FAA3E0FB12187D900146122028900146DD
:102DCF00E0FCA3E0FDA3E0FEA3E0FFC004C005C04C
:102DDF0006C0077F007E007D007C40900142E0F836
:102DEF00A3E0F9A3E0FAA3E0FB12196E125A617B7C
:102DFF00D57A7879E9783D12196EC004C005C006FE
:102E0F00C0077F007E007D007C40900136E0F8A374
:102E1F00E0F9A3E0FAA3E0FB12196E125A617BD11D
:102E2F007A22795B783E12196ED003D002D001D08E
:102E3F0000121879C004C005C006C0077F007E00CD
:102E4F007D007C4090013EE0F8A3E0F9A3E0FAA3F7
:102E5F00E0FB12196EC004C005C006C0077F007EDC
:102E6F00007D007C40900136E0F8A3E0F9A3E0FA82
:102E7F00A3E0FB12196ED003D002D001D0001218BC
:102E8F0079125A617BFC7AA97971783D12196EA873
:102E9F0004A905AA06AB07D007D006D005D00412A7
:102EAF001879C004C005C006C0077F007E007D00F2
:102EBF007C4090013EE0F8A3E0F9A3E0FAA3E0FB29
:102ECF0012196EC004C005C006C00790013AE0FC9D
:102EDF00A3E0FDA3E0FEA3E0FF900136E0F8A3E03E
:102EEF00F9A3E0FAA3E0FB12187DD003D002D001C2
:102EFF00D000121879125A617BD57A787969783DAA
:102F0F0012196EA804A905AA06AB07D007D006D0E0
:102F1F0005D0041218799001E2E0F8A3E0F9A3E0DC
:102F2F00FAA3E0FB12196EA804A905AA06AB07D0F5
:102F3F0007D006D005D00412187D90014612202824
:102F4F007F007E007D007C4090013EE0F8A3E0F919
:102F5F00A3E0FAA3E0FB12196E125A617BE37AC762
:102F6F007928783F12196EC004C005C006C00790BB
:102F7F000136E0FCA3E0FDA3E0FEA3E0FF125A61DF
:102F8F007B9E7A5E79C7784012196EA804A905AAAC
:102F9F0006AB07D007D006D005D00412187DC004A9
:102FAF00C005C006C0077F007E007D007C409001F9
:102FBF003EE0F8A3E0F9A3E0FAA3E0FB12196EA834
:102FCF0004A905AA06AB07900136E0FCA3E0FDA318
:102FDF00E0FEA3E0FF121879125A617BE57AD079EF
:102FEF00A2783F12196EA804A905AA06AB07D0074D
:102FFF00D006D005D0041218799001E2E0F8A3E0D2
:10300F00F9A3E0FAA3E0FB12196E900142E0F8A3D6
:10301F00E0F9A3E0FAA3E0FB12187D90014A122019
:10302F00287F007E007D007C4090013EE0F8A3E009
:10303F00F9A3E0FAA3E0FB12196EA804A905AA06EA
:10304F00AB07900142E0FCA3E0FDA3E0FEA3E0FF8D
:10305F00121879125A617B067A817915783E121906
:10306F006EC004C005C006C00790014AE0FCA3E093
:10307F00FDA3E0FEA3E0FF125A617BA67A9B79A421
:10308F00784012196ED003D002D001D000121879F7
:10309F009001E2E0F8A3E0F9A3E0FAA3E0FB121934
:1030AF006E90014E122028900146E0FCA3E0FDA394
:1030BF00E0FEA3E0FF125A61C004C005C006C007BE
:1030CF0090014EE0FCA3E0FDA3E0FEA3E0FF125A47
:1030DF004BA804A905AA06AB07D007D006D005D088
:1030EF000412196E7B327AAF79CB783E12196EC00B
:1030FF0004C005C006C00790014EE0FCA3E0FDA38D
:10310F00E0FEA3E0FF125A617BDB7ADE796A783F3B
:10311F0012196EA804A905AA06AB07D007D006D0CE
:10312F0005D00412187D900123E0FBA3E0FAA3E081
:10313F00F9121FB6900123E0FBA3E0FAA3E0F91206
:10314F001F96900123E0FBA3E0FAA3E0F9122008F9
:10315F0012196EA804A905AA06AB077F007E007D91
:10316F00807C3F1218791267D09000E812202890C7
:10317F000123E0FBA3E0FAA3E0F9121F96126A5CA9
:10318F00900123E0FBA3E0FAA3E0F9121FB6900130
:10319F0046E0FCA3E0FDA3E0FEA3E0FF125A4BC004
:1031AF0004C005C006C00790014EE0FCA3E0FDA3DC
:1031BF00E0FEA3E0FF125A4BA804A905AA06AB072D
:1031CF00D007D006D005D00412196EC004C005C0B8
:1031DF0006C007900123E0FBA3E0FAA3E0F9121F5A
:1031EF0096125A4BA804A905AA06AB07D007D0061A
:1031FF00D005D004121A7790015212202890014660
:10320F00E0FCA3E0FDA3E0FEA3E0FF125A61C004BF
:10321F00C005C006C00790014EE0FCA3E0FDA3E08F
:10322F00FEA3E0FF125A4BA804A905AA06AB07D0CC
:10323F0007D006D005D00412196E7BDB7ADE796ACF
:10324F00783F12196EC004C005C006C00790014E2A
:10325F00E0FCA3E0FDA3E0FEA3E0FF125A617B3286
:10326F007AAF79CB783E12196EA804A905AA06ABDE
:10327F0007D007D006D005D004121879C004C005B6
:10328F00C006C007900123E0FBA3E0FAA3E0F91208
:10329F001F96125A4BA804A905AA06AB07D007D050
:1032AF0006D005D004121A779001561220289001EB
:1032BF0056E0FCA3E0FDA3E0FEA3E0FFC004C005C1
:1032CF00C006C007900152E0FCA3E0FDA3E0FEA3FF
:1032DF00E0FF9000E8122028D007D006D005D004D8
:1032EF00126A5C900120E0FBA3E0FAA3E0F9121F41
:1032FF00B6900120E0FBA3E0FAA3E0F9121F967B42
:10330F00007A0079007800121B146030402E900173
:10331F0020E0FBA3E0FAA3E0F9C003C002C0011252
:10332F001F969001E6E0F8A3E0F9A3E0FAA3E0FB13
:10333F0012187DD001D002D003121FB6900120E0E9
:10334F00FBA3E0FAA3E0F9121F969001E6E0F8A3C1
:10335F00E0F9A3E0FAA3E0FB121B14502E9001201A
:10336F00E0FBA3E0FAA3E0F9C003C002C001121F03
:10337F00969001E6E0F8A3E0F9A3E0FAA3E0FB12D0
:0B338F001879D001D002D003121FB645
:01339A002210
:0B4676009001A8EBF0A3EAF0A3E9F02C
:104681009001AEE0FCA3E0FDA3E0FEA3E0FFEC128D
:104691001B927B007A81798878C612187D9001B2CD
:1046A100E0F8A3E0F9A3E0FAA3E0FB12187D7B0098
:1046B1007AAD790E7847121A779001B61220287FC9
:1046C100A67EFE7DC77C429001B6E0F8A3E0F9A387
:1046D100E0FAA3E0FB12196E7B917AEA797E783FCA
:1046E10012187D126E3F9001BA1220287F117E238D
:1046F1007D5F7C379001B6E0F8A3E0F9A3E0FAA36F
:10470100E0FB12196EA804A905AA06AB077F507E2B
:10471100AC7DAE7C3B121879126E3FC004C005C05F
:1047210006C0079001BAE0FCA3E0FDA3E0FEA3E010
:10473100FF125A61A804A905AA06AB07D007D00643
:10474100D005D00412196EC004C005C006C0077F91
:10475100187E017DC87C429001B6E0F8A3E0F9A380
:10476100E0FAA3E0FB12196E7B327AE47946783FD6
:1047710012187D126E3FA804A905AA06AB07D0073F
:10478100D006D005D00412187DC004C005C006C0F3
:10479100077F007E007D007C409001BAE0F8A3E035
:1047A100F9A3E0FAA3E0FB12196E125A617B0C7AAD
:1047B100347969783812196EA804A905AA06AB07DD
:1047C100D007D006D005D00412187D9001BE12206A
:1047D100287F147E6A7D177C389001B6E0F8A3E04B
:1047E100F9A3E0FAA3E0FB12196EA804A905AA0631
:1047F100AB077F6D7E6A7D857C3D121879126E3F15
:104801009001C21220289001BEE0FCA3E0FDA3E0CC
:10481100FEA3E0FF125A9DC004C005C006C0079068
:1048210001C2E0FCA3E0FDA3E0FEA3E0FF125A4BAE
:10483100A804A905AA06AB07D007D006D005D00465
:1048410012196E125BAB9001A8E0FBA3E0FAA3E0A2
:10485100F9121FB69001E6E0F8A3E0F9A3E0FAA38C
:10486100E0FB9001BEE0FCA3E0FDA3E0FEA3E0FFBE
:10487100121A771263119001E6E0F8A3E0F9A3E0C0
:10488100FAA3E0FB12196EA804A905AA06AB0790CA
:1048910001BEE0FCA3E0FDA3E0FEA3E0FF12187956
:1048A1009001C61220287F007E007DC07C3F9001D0
:1048B100EAE0F8A3E0F9A3E0FAA3E0FB12196E9095
:1048C10001C6E0F8A3E0F9A3E0FAA3E0FB121B1490
:1048D100505A7F007E007D007C3F9001EAE0F8A302
:1048E100E0F9A3E0FAA3E0FB12196E9001C6E0F82B
:1048F100A3E0F9A3E0FAA3E0FB121B14402E900100
:10490100A8E0FBA3E0FAA3E0F9C003C002C00112D2
:104911001F969001EAE0F8A3E0F9A3E0FAA3E0FB17
:1049210012187DD001D002D003121FB69001A8E069
:10493100FBA3E0FAA3E0F9C003C002C001121F9675
:10494100C004C005C006C0079001A8E0FBA3E0FABF
:10495100A3E0F9121F969001E6E0F8A3E0F9A3E0C5
:10496100FAA3E0FB121A771263119001E6E0F8A3B3
:10497100E0F9A3E0FAA3E0FB12196EA804A905AAC5
:1049810006AB07D007D006D005D004121879D001A4
:10499100D002D003121FB69001BEE0FCA3E0FDA33C
:1049A100E0FEA3E0FF125A61C004C005C006C007C3
:1049B1009001C2E0FCA3E0FDA3E0FEA3E0FF125AD8
:1049C10061A804A905AA06AB07D007D006D005D077
:1049D1000412196E9001ABE0FBA3E0FAA3E0F91217
:1049E1001FB69001ABE0FBA3E0FAA3E0F9121F961A
:1049F1009001ABE0FBA3E0FAA3E0F9122008121941
:104A01006EA804A905AA06AB077F007E007D807C05
:104A11003F1218791267D09000E81220289001AB5C
:104A2100E0FBA3E0FAA3E0F9121F96126A5C900181
:0C4A3100ABE0FBA3E0FAA3E0F9121FB613
:014A3D002256
:0B339B00900182EBF0A3EAF0A3E9F040
:1033A6007F927E0A7D867C3E900188E0F8A3E0F954
:1033B600A3E0FAA3E0FB12196E90018CE0F8A3E0FB
:1033C600F9A3E0FAA3E0FB121879900194122028E1
:1033D6007F007E007D007C00900194E0F8A3E0F978
:1033E600A3E0FAA3E0FB121B145027900194E0FC23
:1033F600A3E0FDA3E0FEA3E0FF9001E6E0F8A3E072
:10340600F9A3E0FAA3E0FB12187D9001941220289C
:1034160080489001E6E0FCA3E0FDA3E0FEA3E0FF08
:10342600900194E0F8A3E0F9A3E0FAA3E0FB121BF5
:103436001460274025900194E0FCA3E0FDA3E0FE84
:10344600A3E0FF9001E6E0F8A3E0F9A3E0FAA3E029
:10345600FB121879900194122028900194E0F8A3A9
:10346600E0F9A3E0FAA3E0FB90001EE0FCA3E0FD78
:10347600A3E0FEA3E0FF1218799000161220289010
:103486000016E0FCA3E0FDA3E0FEA3E0FF125A4B0A
:10349600C004C005C006C00790001AE0FCA3E0FD0A
:1034A600A3E0FEA3E0FF125A4BA804A905AA06ABA7
:1034B60007D007D006D005D00412196EC004C00587
:1034C600C006C007900190E0FCA3E0FDA3E0FEA3C8
:1034D600E0FF125A4BA804A905AA06AB07D007D0ED
:1034E60006D005D00412196EC004C005C006C00778
:1034F60090001AE0FCA3E0FDA3E0FEA3E0FF125A51
:1035060061C004C005C006C007900190E0FCA3E0BE
:10351600FDA3E0FEA3E0FF125A61A804A905AA06CE
:10352600AB07D007D006D005D00412196EA804A99F
:1035360005AA06AB07D007D006D005D00412187D21
:10354600900198122028900198E0FCA3E0FDA3E0EA
:10355600FEA3E0FF900198E0F8A3E0F9A3E0FAA348
:10356600E0FB12196EA804A905AA06AB077F007E28
:10357600007D807C3F1218791267D090019C122042
:1035860028900198E0FCA3E0FDA3E0FEA3E0FFC0C5
:1035960004C005C006C00790019CE0FCA3E0FDA3A3
:1035A600E0FEA3E0FF9000E8122028D007D006D066
:1035B60005D004126A5C900185E0FBA3E0FAA3E063
:1035C600F9121FB6900185E0FBA3E0FAA3E0F91219
:1035D6001F96125A4BC004C005C006C0079001854D
:1035E600E0FBA3E0FAA3E0F9121F96125A61D0039A
:1035F600D002D001D000121A77C004C005C006C0A0
:103606000790001AE0FCA3E0FDA3E0FEA3E0FF1292
:103616005A4BC004C005C006C00790001AE0FCA3C0
:10362600E0FDA3E0FEA3E0FF125A61D003D002D072
:1036360001D000121A77A804A905AA06AB07D0077D
:10364600D006D005D00412196EC004C005C006C04D
:1036560007900185E0FBA3E0FAA3E0F9121F96129A
:103666005A4BC004C005C006C00790001AE0FCA370
:10367600E0FDA3E0FEA3E0FF125A4BA804A905AAA9
:1036860006AB07D007D006D005D00412196EC004C9
:10369600C005C006C007900190E0FCA3E0FDA3E0D2
:1036A600FEA3E0FF125A61D003D002D001D000126F
:1036B6001A77D003D002D001D0001218799001A455
:1036C600122028900190E0FCA3E0FDA3E0FEA3E019
:1036D600FF125A4BC004C005C006C00790001AE08E
:1036E600FCA3E0FDA3E0FEA3E0FF125A4BA804A949
:1036F60005AA06AB07D007D006D005D00412196E6E
:10370600C004C005C006C007900016E0FCA3E0FD9B
:10371600A3E0FEA3E0FF125A4BA804A905AA06AB34
:1037260007D007D006D005D00412196EC004C00514
:10373600C006C007900190E0FCA3E0FDA3E0FEA355
:10374600E0FF125A61C004C005C006C00790001A07
:10375600E0FCA3E0FDA3E0FEA3E0FF125A61A8048B
:10376600A905AA06AB07D007D006D005D0041219C2
:103776006EA804A905AA06AB07D007D006D005D0C7
:103786000412187D9001A0122028900190E0FCA35D
:10379600E0FDA3E0FEA3E0FF125A4BC004C005C043
:1037A60006C007900016E0FCA3E0FDA3E0FEA3E040
:1037B600FF125A61A804A905AA06AB07D007D006CE
:1037C600D005D00412196EC004C005C006C007900B
:1037D60001A0E0FCA3E0FDA3E0FEA3E0FF9001A0B2
:1037E600E0F8A3E0F9A3E0FAA3E0FB12196EA8043F
:1037F600A905AA06AB077F007E007D807C3F1218D4
:10380600791267D0A804A905AA06AB07D007D00687
:10381600D005D004121A779001A01220289001A09A
:10382600E0FCA3E0FDA3E0FEA3E0FFC004C005C0EA
:1038360006C0079001A4E0FCA3E0FDA3E0FEA3E020
:10384600FF9000E8122028D007D006D005D0041239
:103856006A5C900182E0FBA3E0FAA3E0F9121FB6CE
:10386600900182E0FBA3E0FAA3E0F9121F967B0029
:103876007A0079007800121B146030402E90018285
:10388600E0FBA3E0FAA3E0F9C003C002C001121FE7
:10389600969001E6E0F8A3E0F9A3E0FAA3E0FB12B4
:0B38A600187DD001D002D003121FB625
:0138B10022F4
:10672000323B171C0205006400640001000007A34F
:106730000087038400640708038406820569000754
:1067400000020009003B003B0017001C000C006326
:1067500000C700C70002000A0E0F03840E0F038457
:106760000E0F07080E0F070800080007000E0000B4
:106770000000000000010001000000010001000015
:106780000000000000000000000000000000000009
:1067900000000000000000000000000300000003F3
:1067A00000020003000200030003000200030002D5
:1067B00000030000000300010003000200030002C8
:0C67C000000300030002000300020003BD
:066DC700C119C11BC11A35
:106B93009000107432F0900011743BF09000127466
:106BA30017F0900013741CF09000147402F090001E
:106BB300157405F0125038757900757A00D3E57AAB
:106BC300940EE57964809480503CE57A25E0FFE5F6
:106BD3007933FE74262FF58274673EF583E493FCC4
:106BE300740193FDE57A25E0FFE57933FE74222FE6
:106BF300F58274003EF583ECF0A3EDF0057AE57AB7
:106C03007002057980B712513C900068E4F0A3E468
:106C1300F090006AE4F0A3E4F090006CE4F0A3E4E5
:056C2300F012515E2299
:10422B0090003FE0F574D3E57464809482400BC337
:10423B00E574648094865002C219E5A064FFFFEF19
:10424B005407F576E5766006C29CC2988002D29C34
:10425B00E5765406FFEF60270578E578D3940A409E
:10426B000F75750AC3E57464809486500375780ADC
:10427B00E578D39414400E757564757814800675C3
:10428B007800757501AF74EF3395E0FEEF25E0FF15
:10429B00EE33FE746E2FF58274673EF583E493F56F
:1042AB0072740193F573AF74EF3395E0FEEF25E075
:1042BB00FFEE33FE74442FF58274673EF583E4936F
:1042CB00F570740193F571E5746403706B900015D0
:1042DB00E0FFEF75F004121E50AFF0EF602E900070
:1042EB0014E0FFEF3395E0FEEF25E0FFEE33FE74B5
:1042FB00982FF58274673EF583E493FE740193FF68
:10430B00EF2571F571EE3570F570802C900014E08F
:10431B00FFEF3395E0FEEF25E0FFEE33FE74B22F97
:10432B00F58274673EF583E493FE740193FFEF25EA
:10433B0071F571EE3570F570E576B40110900028CB
:10434B00E0FEA3E0FFEF4E70040577800375770066
:10435B00E577C394144008757700A219B39219D36B
:10436B00E57664809481500302461AC3E574648039
:10437B009486400302444012508DE57664047055D8
:10438B00AF74EF3395E0FE74102FF58274003EF599
:10439B0083E02575F0AF74EF3395E0FE74102FF5C5
:1043AB008274003EF583E0FFEF3395E0FED3EF958B
:1043BB0071E5706480F8EE6480984016AF73AE744C
:1043CB00EEFD3395E0FC74102DF58274003CF58303
:1043DB00EFF0125038E5766402705AAF74EF3395F4
:1043EB00E0FE74102FF58274003EF583E0FFC3EFFF
:1043FB009575FFEFF0AF74EF3395E0FE74102FF56A
:10440B008274003EF583E0FFEF3395E0FEC3EF953A
:10441B0073E5726480F8EE6480985016AF71AE74D9
:10442B00EEFD3395E0FC74102DF58274003CF583A2
:10443B00EFF0125038C3E574648094865003024544
:10444B005C74FA2574F574E57664047072AF75EFDD
:10445B00FD7C00AF74EF3395E0FEEF25E0FFEE330C
:10446B00FE74222FF58274003EF583EC8DF0121F43
:10447B0012AF74EF3395E0FEEF25E0FFEE33FE74E1
:10448B00222FF58274003EF583E0FEA3E0FFD3EF0D
:10449B009571E5706480F8EE648098401FAF74EFFF
:1044AB003395E0FEEF25E0FFEE33FE74222FF5820D
:1044BB0074003EF583E572F0A3E573F012513CE511
:1044CB007664026003024556AF74EF3395E0FEEF5E
:1044DB0025E0FFEE33FE74222FF58274003EF58348
:1044EB00C083C082E0FEA3E0FFAD757C00C3EF9DEF
:1044FB00FFEE9CFED082D083EEF0A3EFF0AF74EF13
:10450B003395E0FEEF25E0FFEE33FE74222FF582AC
:10451B0074003EF583E0FEA3E0FFC3EF9573E572F5
:10452B006480F8EE648098501FAF74EF3395E0FE13
:10453B00EF25E0FFEE33FE74222FF58274003EF57B
:10454B0083E570F0A3E571F012513C74062574F508
:10455B0074900028E0FEA3E0FFEF4E705CE576B4AC
:10456B000526301B230574AF74D3EF6480949340FE
:10457B0003757400C21BAF74EF3395E0FE90003EE1
:10458B00EEF0A3EFF012513CE576640360030246B4
:10459B001A301B7B1574AF74C3EF64809480500387
:1045AB00757413C21BAF74EF3395E0FE90003EEEB3
:1045BB00F0A3EFF012513C8056E576B40526301B84
:1045CB00230574AF74D3EF64809492400375740029
:1045DB00C21BAF74EF3395E0FE90003EEEF0A3EFFD
:1045EB00F012513CE576B40326301B231574AF74DF
:1045FB00C3EF648094805003757412C21BAF74EFC9
:10460B003395E0FE90003EEEF0A3EFF012513CE547
:10461B0076B40102D21BE5765406FFEF60109000D2
:10462B003EE0FEA3E0FFEF64094E7002C20F900262
:10463B0005E0FEA3E0FF900028E0FCA3E0FDED6F9A
:10464B007002EC6E6002C20F900028E0FEA3E0FF48
:10465B00900205EEF0A3EFF030A302D21A20A30ACA
:0A466B00301A07C21AA20FB3920F13
:014675002222
:105038001251A774A01251BF74021251BF900010F0
:105048007C03E01251801251BFA3DCF6E0125180BC
:10505800F5F0A3A3E0030354C045F01251BF90003C
:1050680014E01251801251BFC2B412519A1251A7C2
:1050780074A01251BF74F01251BFA3E01251BFC205
:10508800B412519A221251A774A01251BF7402127D
:1050980051BF1251A774A0041251BF9000101251B1
:1050A800E4125188F0A31251F71251E4125188F01A
:1050B800A31251F71251E4125188F0A31251F712BA
:1050C80051E4FB543F125188F0A31251F71251E4F6
:1050D800FA541F125188F0EB23235403FD1251F1A7
:1050E800C2B412519A1251A774A01251BF74F0128F
:1050F80051BF1251A774A0041251BF1251E4FB54BE
:1051080003C39D2405838007030201000302012BCA
:10511800A3F0F5F01251F1C2B412519A1251A774CA
:10512800A01251BF74F01251BFE5F01251BFC2B4C2
:1051380012519A227AA07B807C1E9000221252374C
:10514800227AA07B801251FFED900022F07AA0A372
:105158007C1D12526C227AA07BD07C1090006812C1
:105168005237227AA07BD01251FFED900068F07A76
:01517800A096
:10517900A37C0F12526C2275F00A84C425F022C058
:10518900E0C4540F75F00AA4F5F0D0E0540F25F0EF
:105199002200D2B5000000D2B40000000022125152
:1051A9009AC2B4000000C2B500000022D2B50000C6
:1051B90000C2B50000227E083392B41251B5DEF860
:1051C90033D2B40000A2B450040000A2B41251B505
:1051D900400122C2B4000012519A227E08A2B433BF
:1051E900001251B5DEF7C322D2B41251B522C2B4AE
:1051F9001251B5D2B4221251A7EA1251BFEB125182
:10520900BF1251A7EA041251BF1251E4FD1251F124
:10521900C2B412519A221251A7EA1251BFEB12518C
:10522900BFE61251BF08DCF9C2B412519A221251D9
:10523900A7EA1251BFEB1251BFE01251BFA3DCF92B
:10524900C2B412519A221251A7EA041251BF800323
:105259001251F71251E4F608DCF61251F1C2B412F8
:10526900519A221251A7EA041251BF80031251F731
:0C5279001251E4F0A3DCF61251F1C2B4B3
:0452850012519A2206
:104D3E00202020202531642E25303264202530326B
:104D4E0062753A25303262753A253032627520200E
:104D5E0020200020202020253032642E2531642092
:104D6E0025303262753A25303262753A253032621C
:104D7E00752020202000253033642E25316420201C
:104D8E00253032642E25316420415A2F454C312076
:104D9E00202000253033642E25316420202530322A
:104DAE00642E25316420415A2F454C32202020009C
:104DBE00253033642E2531642020253032642E2593
:104DCE0031642052412F44454320202000253033AA
:104DDE00642E2531645720253032642E2531644EE1
:104DEE00204C4F2F4C412020200025303262752060
:104DFE0020202530326275202025303262753A250A
:104E0E00303262753A25303262752020202000251E
:104E1E0030352E31662020253032642E2531642027
:104E2E0020202020202025303264202000202B2519
:104E3E003031642E2530316420202B253031642E04
:104E4E002530316420434F52202053545020002DE2
:104E5E002D2D2D2D2D2D2D2D2D2D202020202020C2
:104E6E005354502000253033642E253164202025E4
:104E7E003032642E25316420414E54202025316479
:104E8E002E2531642000202020204F204520352063
:104E9E004A2046204C2020202020002020202020A8
:104EAE00202020454D45202020202020202020009D
:104EBE0020416E74656E6E6120436F6E74726F6CFE
:104ECE006C65722000202020202020207620382E95
:104EDE00312020202020202020002020204A414E5A
:104EEE004645424D41524150524D41594A554E4A06
:104EFE00554C4155475345504F43544E4F564445DC
:104F0E0043004D4F4F4E202053554E2020204341FD
:104F1E005353494F4359474E5553534147495454A0
:104F2E005441555255534C454F2020204151554127
:104F3E00522E52412F444543415A2F454C32415A2D
:104F4E002F454C3100326D3A37303A32333A3133E5
:104F5E003A39636D36636D31304732344700205332
:104F6E00534920313062697428373230292020208D
:104F7E002020205353493131626974283138303042
:104F8E002920202020202053534931326269742871
:104F9E003336303029202020202020484831365406
:104FAE0020616E6420496E6B6C2E202020202041E3
:104FBE00322D532D5320313220626974202020204F
:104FCE00202048483136545F3130626974313032B6
:104FDE0034202020202048483136545F3131626918
:104FEE007432303438202020202048483136545F27
:104FFE0031326269743430393620202020204D4100
:10500E004232385F313262697434303936202020B2
:10501E002020000F0C09010306171D664C0309031F
:0A502E0009030903095601010204F9
:10002E00E57664016003125D73201403020663C259
:10003E001430190C900028E0FEA3E0FFEF4E601183
:10004E0090003EE0FEA3E0FFEF64134E600302015A
:10005E00FB90003CE0FEA3E0FFC3EF9404EE64804F
:10006E0094804003020108AF1CAE1B126F00EF24F8
:10007E0005FFEE3400FE7C007D0A121EDC9000E0CF
:10008E00EEF0A3EFF07B017A007980C003C002C0CE
:10009E00017BFF7A4D793E9000F3EBF0A3EAF0A3DB
:1000AE00E9F09000E0E0FEA3E0FF7C007D64121E0C
:1000BE00DC9000F6EEF0A3EFF09000E0E0FEA3E09F
:1000CE00FF7C007D64121EDC9000F8ECF0A3EDF0D6
:1000DE00900012E0FF9000FAEFF0900011E0FF9018
:1000EE0000FBEFF0900010E0FF9000FCEFF0D0016D
:1000FE00D002D003123E0D020198AF1CAE1B126F40
:10010E0000EF2405FFEE3400FE7C007D0A121EDC9B
:10011E009000E0EEF0A3EFF07B017A007980C0034F
:10012E00C002C0017BFF7A4D79619000F3EBF0A322
:10013E00EAF0A3E9F09000E0E0FEA3E0FF7C007D92
:10014E000A121EDC9000F6EEF0A3EFF09000E0E055
:10015E00FEA3E0FF7C007D0A121EDC9000F8ECF09E
:10016E00A3EDF0900012E0FF9000FAEFF090001176
:10017E00E0FF9000FBEFF0900010E0FF9000FCEF2E
:10018E00F0D001D002D003123E0D751500D3E51547
:10019E00648094825042AF1590003DE0FE75F003EE
:1001AE00EEA4F58285F083E5822FF582E43583F5A2
:1001BE0083E5822453F582E583344FF583E493FF80
:1001CE00AE15EEFD3395E0FC74802DF58274003C87
:1001DE00F583EFF0051580B5C3E51B648094804070
:1001EE00030205F3900083742DF00205F390003E98
:1001FE00E0FEA3E0FFEF640A4E601190003EE0FEC9
:10020E00A3E0FFEF640B4E600302029F7B017A00B6
:10021E007980C003C002C0017BFF7A4D79849000C3
:10022E00F3EBF0A3EAF0A3E9F090002AE0FEA3E0DE
:10023E00FF7C007D0A121EDC9000F6EEF0A3EFF0BC
:10024E0090002AE0FEA3E0FF7C007D0A121EDC90E7
:10025E0000F8ECF0A3EDF090002CE0FEA3E0FF7CA4
:10026E00007D0A121EDC9000FAEEF0A3EFF0900073
:10027E002CE0FEA3E0FF7C007D0A121EDC9000FC49
:10028E00ECF0A3EDF0D001D002D003123E0D02052A
:10029E00F390003EE0FEA3E0FFEF640C4E60119081
:1002AE00003EE0FEA3E0FFEF640D4E600302034349
:1002BE007B017A007980C003C002C0017BFF7A4DBA
:1002CE0079A19000F3EBF0A3EAF0A3E9F090002EF1
:1002DE00E0FEA3E0FF7C007D0A121EDC9000F6EE2D
:1002EE00F0A3EFF090002EE0FEA3E0FF7C007D0A6D
:1002FE00121EDC9000F8ECF0A3EDF0900030E0FE62
:10030E00A3E0FF7C007D0A121EDC9000FAEEF0A343
:10031E00EFF0900030E0FEA3E0FF7C007D0A121E9D
:10032E00DC9000FCECF0A3EDF0D001D002D0031273
:10033E003E0D0205F390003EE0FEA3E0FFEF640EDB
:10034E004E601190003EE0FEA3E0FFEF640F4E60A2
:10035E0003020426900034E0FEA3E0FFEF247CFFAE
:10036E00EE34FCFE90007CEEF0A3EFF090007CE00B
:10037E00FEA3E0FF126F007C007D0A121EDCC00699
:10038E00C00790007CE0FEA3E0FF126F007C007DB2
:10039E000A121EDC9000FCECF0A3EDF0D007D006A4
:1003AE009000FAEEF0A3EFF07B017A007980C003A3
:1003BE00C002C0017BFF7A4D79BE9000F3EBF0A333
:1003CE00EAF0A3E9F0900032E0FEA3E0FF7C007DAE
:1003DE000A121EDC9000F6EEF0A3EFF0900032E071
:1003EE00FEA3E0FF7C007D0A121EDC9000F8ECF00C
:1003FE00A3EDF0D001D002D003123E0D90007CE0B0
:10040E00FEA3E0FFC3EE6480948040030205F390E8
:10041E000086742DF00205F390003EE0FEA3E0FF8F
:10042E00EF64104E601190003EE0FEA3E0FFEF641B
:10043E00114E600302054D900036E0FEA3E0FFEF83
:10044E0024F8FFEE34F8FE90007EEEF0A3EFF0906D
:10045E000038E0FEA3E0FFEF247CFFEE34FCFE90BC
:10046E00007CEEF0A3EFF090007EE0FEA3E0FF1222
:10047E006F007C007D0A121EDCC006C00790007E55
:10048E00E0FEA3E0FF126F007C007D0A121EDCC0AE
:10049E0004C00590007CE0FEA3E0FF126F007C001C
:1004AE007D0A121EDCC006C00790007CE0FEA3E0B1
:1004BE00FF126F007C007D0A121EDC9000FCECF037
:1004CE00A3EDF0D007D0069000FAEEF0A3EFF0D037
:1004DE0005D0049000F8ECF0A3EDF0D007D0069014
:1004EE0000F6EEF0A3EFF07B017A007980C003C036
:1004FE0002C0017BFF7A4D79DB9000F3EBF0A3EAAB
:10050E00F0A3E9F0D001D002D003123E0D90007E90
:10051E00E0FEA3E0FFC3EE64809480500690008559
:10052E007445F090007CE0FEA3E0FFC3EE6480947F
:10053E008040030205F390008B7453F00205F37BA9
:10054E00017A007980C003C002C0017BFF7A4D7929
:10055E00F89000F3EBF0A3EAF0A3E9F0900013E0BB
:10056E00FF9000F6EFF0900015E0FF9000F7EFF02F
:10057E00900012E0FF9000F8EFF0900011E0FF9075
:10058E0000F9EFF0900010E0FF9000FAEFF0D001CC
:10059E00D002D003123E0D751500D3E5156480947C
:1005AE00825042AF15900014E0FE75F003EEA4F5F4
:1005BE008285F083E5822FF582E43583F583E5822B
:1005CE0024E8F582E583344EF583E493FFAE15EE11
:1005DE00FD3395E0FC74822DF58274003CF583EFBB
:1005EE00F0051580B5900028E0FEA3E0FFC3EF9460
:1005FE0002EE64809480503290003EE0FEA3E0FF55
:10060E00C3EF940AEE64809480401390003EE0FEA7
:10061E00A3E0FFD3EF9411EE64809480400C900021
:10062E00927444F09000937445F07F00125D8575CE
:10063E001500D3E51564809493501AAF15EF3395DA
:10064E00E0FE74802FF58274003EF583E0FF125DAC
:10065E004C051580DD201503020879C21590003E69
:10066E00E0FEA3E0FFC3EF940AEE64809480401591
:10067E0090003EE0FEA3E0FFD3EF9411EE64809471
:10068E00805002C2199001E2E0F8A3E0F9A3E0FA6B
:10069E00A3E0FB900004E0FCA3E0FDA3E0FEA3E0DA
:1006AE00FF121A77126F787B007A00792078411248
:1006BE00196E7B007A007900783F12187D121BD0DC
:1006CE0090007CEEF0A3EFF09001E2E0F8A3E0F9E9
:1006DE00A3E0FAA3E0FB900078E0FCA3E0FDA3E02A
:1006EE00FEA3E0FF121A77126F787B007A00790072
:1006FE00783F12187D121BD09000E2EEF0A3EFF0BF
:10070E007B017A007998C003C002C0017BFF7A4E4C
:10071E00791D9000F3EBF0A3EAF0A3E9F09001E26B
:10072E00E0F8A3E0F9A3E0FAA3E0FB90000CE0FCF4
:10073E00A3E0FDA3E0FEA3E0FF121A779000F612ED
:10074E00202890007CE0FEA3E0FF7C007D0A121EB4
:10075E00DC9000FAEEF0A3EFF090007CE0FEA3E058
:10076E00FF7C007D0A121EDC9000FCECF0A3EDF085
:10077E009000E2E0FEA3E0FF9000FEEEF0A3EFF0AB
:10078E00D001D002D003123E0D7F007E007D007C92
:10079E0000900004E0F8A3E0F9A3E0FAA3E0FB1256
:1007AE001B14500690009E742DF0751500D3E515A0
:1007BE00648094855042AF15900029E0FE75F006D6
:1007CE00EEA4F58285F083E5822FF582E43583F57C
:1007DE0083E5822410F582E583344FF583E493FF9D
:1007EE00AE15EEFD3395E0FC74A42DF58274003C3D
:1007FE00F583EFF0051580B5900028E0FEA3E0FF2D
:10080E00C3EF9402EE64809480400E9000AA742090
:10081E00F09000AB7420F080217F007E007D007C84
:10082E0000900078E0F8A3E0F9A3E0FAA3E0FB1251
:10083E001B1450069000A9742DF0E5766401602B10
:10084E007F40125D85751500D3E515648094935035
:10085E001AAF15EF3395E0FE74982FF58274003EB3
:10086E00F583E0FF125D4C051580DD2016030209AD
:10087E00CAC216900022E0FEA3E0FFEF249CFFEE1A
:10088E0034FFFE126F0090007EEEF0A3EFF09000AA
:10089E0024E0FEA3E0FFEF249CFFEE34FFFE126F78
:1008AE000090007CEEF0A3EFF03010030209417BC4
:1008BE00017A0079B0C003C002C0017BFF7A4E7985
:1008CE003B9000F3EBF0A3EAF0A3E9F090007EE09A
:1008DE00FEA3E0FF7C007D0A121EDC9000F6EEF017
:1008EE00A3EFF090007EE0FEA3E0FF7C007D0A12F5
:1008FE001EDC9000F8ECF0A3EDF090007CE0FEA37F
:10090E00E0FF7C007D0A121EDC9000FAEEF0A3EFF1
:10091E00F090007CE0FEA3E0FF7C007D0A121EDC5E
:10092E009000FCECF0A3EDF0D001D002D003123E0B
:10093E000D80267B017A0079B0C003C002C0017B16
:10094E00FF7A4E795D9000F3EBF0A3EAF0A3E9F0A5
:10095E00D001D002D003123E0D900022E0FEA3E0A3
:10096E00FFC3EF9464EE6480948050069000B174DF
:10097E002DF0900024E0FEA3E0FFC3EF9464EE643C
:10098E0080948050069000B7742DF0E57664016077
:10099E002B7F14125D85751500D3E5156480949335
:1009AE00501AAF15EF3395E0FE74B02FF582740038
:1009BE003EF583E0FF125D4C051580DD2017030226
:1009CE000BE3C217900027E0FFEF90503593FFEF37
:1009DE003395E0FEAC66AD67121ECA8E4A8F4B9001
:1009EE0001F9E0FEA3E0FF126F007C007D0A121EEB
:1009FE00DCC006C0079001F9E0FEA3E0FF126F0015
:100A0E007C007D0A121EDC9000FCECF0A3EDF0D011
:100A1E0007D0069000FAEEF0A3EFF07B017A007992
:100A2E00C8C003C002C0017BFF7A4E79739000F3F9
:100A3E00EBF0A3EAF0A3E9F09001FBE0FEA3E0FFE8
:100A4E007C007D0A121EDC9000F6EEF0A3EFF09013
:100A5E0001FBE0FEA3E0FF7C007D0A121EDC90008D
:100A6E00F8ECF0A3EDF0AE4AAF4B7C007D0A121EFF
:100A7E00DC9000FEEEF0A3EFF0AE4AAF4B7C007DB3
:100A8E000A121EDC900100ECF0A3EDF0D001D002B2
:100A9E00D003123E0D9001F9E0FEA3E0FFC3EE6419
:100AAE0080948050069000CE742DF0A21CB3921C40
:100ABE00E508540CFFEFB40808201C059000D8E49C
:100ACE00F0E508540CFFEFB40409201C069000D882
:100ADE007401F0E508540CFFEFB40C09300F0690CA
:100AEE0000D8742AF0E5085403FFEFB40209301C55
:100AFE00069000D77402F0E5085403FFEFB4010925
:100B0E00301C069000D77403F0E5085403FFEFB4D1
:100B1E000309300F069000D7742AF090003EE0FED5
:100B2E00A3E0FFEF64124E6003020BB8751500D3FD
:100B3E00E515648094935042AF1590003BE0FE752E
:100B4E00F014EEA4F58285F083E5822FF582E4356C
:100B5E0083F583E582246CF582E583344FF583E4D7
:100B6E0093FFAE15EEFD3395E0FC74C82DF582743F
:100B7E00003CF583EFF0051580B5AE4AAF4B7C0017
:100B8E007D0A121EDCEF2430FF9000D9EFF09000AA
:100B9E00DA742EF0AE4AAF4B7C007D0A121EDCAF2B
:100BAE0005EF2430FF9000DBEFF07F54125D85756A
:100BBE001500D3E51564809493501AAF15EF339555
:100BCE00E0FE74C82FF58274003EF583E0FF125DDF
:100BDE004C051580DDE576B4011490003FE0FFEF83
:100BEE0090502193FF125D85125D6A125D7C301864
:100BFE0003020D467B017A007980C003C002C0015A
:100C0E007BFF7A4E79949000F3EBF0A3EAF0A3E920
:100C1E00F0D001D002D003123E0D7B017A007998FC
:100C2E00C003C002C0017BFF7A4E79A99000F3EB9E
:100C3E00F0A3EAF0A3E9F0D001D002D003123E0DEA
:100C4E007B017A0079B0C003C002C0017BFF7A4EEF
:100C5E0079BE9000F3EBF0A3EAF0A3E9F0D001D057
:100C6E0002D003123E0D7B017A0079C8C003C00288
:100C7E00C0017BFF7A4E79D39000F3EBF0A3EAF03C
:100C8E00A3E9F0D001D002D003123E0D7F00125D19
:100C9E0085751500D3E51564809493501AAF15EF42
:100CAE003395E0FE74802FF58274003EF583E0FFED
:100CBE00125D4C051580DD7F40125D85751500D3E4
:100CCE00E51564809493501AAF15EF3395E0FE74DA
:100CDE00982FF58274003EF583E0FF125D4C0515EA
:100CEE0080DD7F14125D85751500D3E51564809443
:100CFE0093501AAF15EF3395E0FE74B02FF5827452
:100D0E00003EF583E0FF125D4C051580DD7F541229
:100D1E005D85751500D3E51564809493501AAF1553
:100D2E00EF3395E0FE74C82FF58274003EF583E034
:090D3E00FF125D4C051580DD2259
:106DCD00015100014F00015000014900C10FC10CDC
:0A6DDD00C10BC10EC110C10DC111A0
:106F1200752400D3E524648094A75004052480F3EB
:016F2200224C
:106F2300752500D3E525648094935004052580F3EB
:016F3300223B
:106F3400752600D3E5266480949E5004052680F3CC
:016F4400222A
:106F4500752700D3E5276480949E5004052780F3B8
:016F55002219
:106F5600752800C3E5286480949E5004052880F3B4
:016F66002208
:106F6700752900C3E529648094815004052980F3BD
:016F770022F7
:10621000C292C296126F12126F12C290126F127552
:106220002F1F752E00E52ED394075011E52FC313B1
:10623000F52FA2D79290126F12052E80E8D29012FD
:106240006F12D292752A03752BE8752F00309110CA
:10625000E52B152B7002152A14FFAE2AEF4E70EDB8
:10626000126F23752E00E52ED394075013126F1270
:10627000E52FC313F52F309103432F80052E80E6C1
:10628000126F12AF2F7E00EF752D00F52C752A03CB
:10629000752BE8752F00309110E52B152B7002152A
:1062A0002A14FFAE2AEF4E70ED126F23752E00E513
:1062B0002ED394075013126F12E52FC313F52F300E
:1062C0009103432F80052E80E6126F12AF2F7E00C0
:1062D000EF252DF52DEE352CF52CC3E52C6480949F
:1062E000805006752C00752D00D3E52D940FE52CFC
:1062F0006480948E4006752C0E752D0F20B20DC350
:10630000740F952DF52D740E952CF52CAE2CAF2D0C
:01631000226A
:10640100C294126F1275351F753400E534D39407A9
:106411005011E535C313F535A2D79294126F1205C9
:106421003480E8D294126F12D2967530037531E838
:10643100753500309510E53115317002153014FFB6
:10644100AE30EF4E70ED126F23753400E534D39406
:10645100075013126F12E535C313F5353095034319
:106461003580053480E6126F12AF357E00EF75334B
:1064710000F5327530037531E8753500309510E55A
:106481003115317002153014FFAE30EF4E70ED1240
:106491006F23753400E534D394075013126F12E55E
:1064A10035C313F535309503433580053480E61245
:1064B1006F12AF357E00EF2533F533EE3532F5320D
:1064C100C3E532648094805006753200753300D381
:1064D100E533940FE5326480948E400675320E7573
:0664E100330FAE32AF33B1
:0164E7002292
:10000E001262108E4D8F4E1264018E478F487566A8
:05001E000075670122DE
:10691D00D290D294D291D295756C00756D00756838
:10692D0000756900753600D3E53664809489504949
:10693D00126F34C290C294126F34C3E536648094E2
:10694D00895004D290D294E56D256DF56DE56C35C9
:10695D006CF56CE5692569F569E5683568F56820BC
:10696D009108056DE56D7002056C2095080569E5CA
:10697D006970020568053680AEC290C294756600D6
:10698D00756705AE6CAF6D7C007D05121ECA8E4D10
:10699D008F4E20B20DC3740B954EF54E740E954D62
:1069AD00F54DAE68AF697C007D05121ECA8E478F0E
:0169BD004891
:0169BE0022B6
:106AF900D290D294D291D295756C00756D0075685B
:106B090000756900753700D3E5376480948A504968
:106B1900126F34C290C294126F34C3E53764809403
:106B29008A5004D290D294E56D256DF56DE56C35EA
:106B39006CF56CE5692569F569E5683568F56820DE
:106B49009108056DE56D7002056C2095080569E5EC
:106B59006970020568053780AEC290C294756600F7
:106B6900756702E56D25E0F54EE56C33F54D20B20C
:106B79000DC3740E954EF54E740E954DF54DE569A0
:096B890025E0F548E56833F54705
:016B920022E0
:106CB900D290D294D291D295756C00756D00756899
:106CC90000756900753800D3E5386480948B5049A4
:106CD900126F34C290C294126F34C3E53864809441
:106CE9008B5004D290D294E56D256DF56DE56C3528
:106CF9006CF56CE5692569F569E5683568F568201D
:106D09009108056DE56D7002056C2095080569E52A
:106D19006970020568053880AEC290C29475660034
:106D2900756701856C4D856D4E20B20DC3740F9545
:0F6D39004EF54E740E954DF54D856847856948AA
:016D48002228
:105DCA00D292D291756C00756D00126F45753900CB
:105DDA00D3E5396480948F5025D290126F67C290B0
:105DEA00126F67E56D256DF56DE56C356CF56C2008
:105DFA009108056DE56D7002056C053980D2C29077
:105E0A00C292E56DAE6C7806CEC313CE13D8F9F5FF
:105E1A006D8E6CAC6CAD6DE4121B977B007A0079C9
:105E2A0034784412196E7B007A0079807844121A09
:105E3A0077121BD07C007D05121ECA8E4D8F4E2014
:105E4A00B20DC3740B954EF54E740E954DF54D1269
:105E5A006F45756600756705D296D29575680075A7
:105E6A006900126F45753900D3E5396480948F5003
:105E7A0025D294126F67C294126F67E5692569F596
:105E8A0069E5683568F5682095080569E56970026D
:105E9A000568053980D2C294C296E569AE6878066B
:105EAA00CEC313CE13D8F9F5698E68AC68AD69E430
:105EBA00121B977B007A007934784412196E7B00A2
:105ECA007A0079807844121A77121BD07C007D05FB
:075EDA00121ECA8E478F481B
:015EE100229E
:105EE200D292D291756C00756D00126F45753A00B1
:105EF200D3E53A6480948F5025D290126F67C29096
:105F0200126F67E56D256DF56DE56C356CF56C20EE
:105F12009108056DE56D7002056C053A80D2C2905C
:105F2200C292E56DAE6C7805CEC313CE13D8F9F5E7
:105F32006D8E6CAC6CAD6DE4121B977B007A0079B0
:105F4200E1784412196E7B007A0079007845121AC2
:105F520077121BD0EF25E0F54EEE33F54D20B20D52
:105F6200C3740E954EF54E740E954DF54D126F4558
:105F7200756600756702D296D295756800756900DC
:105F8200126F45753A00D3E53A6480948F5025D25A
:105F920094126F67C294126F67E5692569F569E526
:105FA200683568F5682095080569E5697002056835
:105FB200053A80D2C294C296E569AE687805CEC32E
:105FC20013CE13D8F9F5698E68AC68AD69E4121B7B
:105FD200977B007A0079E1784412196E7B007A008F
:105FE20079007845121A77121BD0EF25E0F548EEBA
:035FF20033F5473D
:015FF5002289
:10610400D292D291756C00756D00126F45753B008B
:10611400D3E53B6480948F5025D290126F67C29070
:10612400126F67E56D256DF56DE56C356CF56C20CA
:106134009108056DE56D7002056C053B80D2C29037
:10614400C292E56CC4F854F0C868F56CE56DC454AB
:106154000F48F56DAC6CAD6DE4121B977B007A00B3
:106164007961784512196E7B007A0079807845123E
:106174001A77121BD08E4D8F4E20B20DC3740F951B
:106184004EF54E740E954DF54D126F4575660075BE
:106194006701D296D295756800756900126F4575CE
:1061A4003B00D3E53B6480948F5025D294126F67F3
:1061B400C294126F67E5692569F569E5683568F584
:1061C400682095080569E56970020568053B80D279
:1061D400C294C296E568C4F854F0C868F568E569E5
:1061E400C4540F48F569AC68AD69E4121B977B0091
:1061F4007A007961784512196E7B007A007980788B
:0B62040045121A77121BD08E478F48FE
:01620F00226C
:105FF600D292D291756C00756D00126F45753C009A
:10600600D3E53C6480948F5025D290126F67C2907E
:10601600126F67E56D256DF56DE56C356CF56C20D9
:106026009108056DE56D7002056C053C80D2C29045
:10603600C292E56CC4F854F0C868F56CE56DC454BA
:106046000F48F56DAC6CAD6DE4121B977B007A00C2
:106056007961784512196E7B007A0079807845124D
:106066001A77121BD08E4D8F4E20B20DC3740F952A
:106076004EF54E740E954DF54D126F4575660075CD
:106086006701D295756800756900126F67753C00E7
:10609600D3E53C6480948C5032C294126F67D294DC
:1060A600D294D294D294D294D294D294D294D294BA
:1060B600E5692569F569E5683568F5682095080597
:1060C60069E56970020568053C80C5D294E568C338
:1060D60013F568E56913F569AC68AD69E4121B97B9
:1060E6007B007A007961784512196E7B007A007917
:0D60F600807845121A77121BD08E478F4814
:016103002279
:10585F00D292D291756C00756D00126F56753D0026
:10586F00D3E53D6480948F5025D290126F56C2902D
:10587F00126F56E56D256DF56DE56C356CF56C2089
:10588F009108056DE56D7002056C053D80D2C290E3
:10589F00C292E56CC4F854F0C868F56CE56DC45459
:1058AF000F48F56DD3E56D9559E56C955840188502
:1058BF006C62856D63856C58856D59E56D24FFF5B8
:1058CF0057E56C34FFF556C3E56D9557E56C955666
:1058DF00501EE56D2401F563E56C3400F562856CAF
:1058EF0056856D57E56D2401F559E56C3400F55873
:1058FF00AC62AD63EC121B977B007A00796178453F
:10590F0012196E7B007A0079807845121A77121B74
:10591F00D08E4D8F4E20B20DC3740F954EF54E7431
:10592F000E954DF54D126F45756600756701D29650
:10593F00D295756800756900126F56753D00D3E5F5
:10594F003D6480948F5025D294126F56C294126F7B
:10595F0056E5692569F569E5683568F568209508A4
:10596F000569E56970020568053D80D2C294C2964B
:10597F00E568C4F854F0C868F568E569C4540F4881
:10598F00F569D3E5699555E5689554401885685EC6
:10599F0085695F856854856955E56924FFF553E589
:1059AF006834FFF552C3E5699553E5689552501E6B
:1059BF00E5692401F55FE5683400F55E8568528579
:1059CF006953E5692401F555E5683400F554AC5E7B
:1059DF00AD5FEC121B977B007A0079617845121945
:1059EF006E7B007A0079807845121A77121BD08E61
:0359FF00478F4887
:015A02002281
:1038B200E54C64326003300D60C3E56F954EF561EF
:1038C200E56E954DF560C374089548FF74079547FA
:1038D200FE126F00EF247CFFEE34FCFEC3E56B9F0B
:1038E200F55BE56A9EF55AC3E5489408E5476480AE
:1038F2009487500BC3E4955BF55BE4955AF55AC285
:1039020010C20E900068E560F0A3E561F090006AD5
:10391200E55AF0A3E55BF0C20D20101B20B3033083
:103922000E03301112D210D20E90006CE4F0A37488
:1039320001F012515EC21130101D20B303300E038C
:10394200301114C210D20E12514990006CE4F0A34F
:10395200E4F012515EC21120B304054C8005754C8F
:1039620000C20E301074E561254EF54EE560354D0E
:10397200F54DD3E54E940FE54D6480948E400C7462
:10398200F0254EF54E74F1354DF54DC3E54D64808D
:103992009480500C7410254EF54E740E354DF54D35
:1039A200E55B2548F548E55A3547F547D3E54894A0
:1039B2000FE5476480948E400C74F02548F54874F6
:1039C200F13547F547C3E54764809480500C741085
:1039D2002548F548740E3547F547C374089548FFE6
:1039E20074079547FE126F00EF247CF548EE34FC15
:1039F200F5479001FBE54DF0A3E54EF09001F9E5A6
:103A020047F0A3E548F0E56F24F8F55DE56E34F87C
:103A1200F55CE54E24F8F565E54D34F8F564C3E54B
:103A22005C64809480500C7410255DF55D740E35D5
:103A32005CF55CC3E56464809480500C7410256569
:103A4200F565740E3564F56430105A900038E0FE66
:103A5200A3E0FFC3EF9484EE64809483400FC3E538
:103A62006F954EF53FE56E954DF53E800DC3E55DD4
:103A72009565F53FE55C9564F53ED3E56B9400E50D
:103A82006A648094804010C3E56B9548F541E56A0D
:103A92009547F540023B4FC3E49548F541E495470D
:103AA200F540023B4F900038E0FEA3E0FFC3EF94E5
:103AB20084EE648094834025900022E0FEA3E0FF20
:103AC200E56F2FFFE56E3EFEEF249CFFEE34FFFE16
:103AD200C3EF954EF53FEE954DF53E8023900022C3
:103AE200E0FEA3E0FFE55D2FFFE55C3EFEEF249CD8
:103AF200FFEE34FFFEC3EF9565F53FEE9564F53EAC
:103B0200D3E56B9400E56A6480948040259000249C
:103B1200E0FEA3E0FFE56B2FFFE56A3EFEEF249C8B
:103B2200FFEE34FFFEC3EF9548F541EE9547F540B1
:103B3200801B900024E0FEA3E0FFEF249CFFEE3404
:103B4200FFFEC3EF9548F541EE9547F54075080F26
:103B5200200F03023D87AE4AAF4B7C007D02121E4E
:103B6200DCD3E53F9FEE6480F8E53E648098402414
:103B7200E54620E5067551007550000551AF51EF3D
:103B8200D394504003755150E551C3940A405053A9
:103B9200080E804BAE4AAF4B7C007D02121EDCC386
:103BA200E49FFFE49EFEC3E53F9FEE6480F8E53E9E
:103BB2006480985024E54620E40675510075500053
:103BC2000551AF51EFD394504003755150E551C3A5
:103BD200940A400B53080D8006755100755000AED3
:103BE2004AAF4B7C007D02121EDCD3E5419FEE649E
:103BF20080F8E5406480984024E54620E706754F4A
:103C020000754900054FAF4FEFD394504003754FF5
:103C120050E54FC3940A405D53080B8058AE4AAF3B
:103C22004B7C007D02121EDCC3E49FFFE49EFEC3B8
:103C3200E5419FEE6480F8E5406480985031D3E519
:103C4200489400E547648094804024E54620E606D7
:103C5200754F00754900054FAF4FEFD394504003A5
:103C6200754F50E54FC3940A400B53080780067501
:103C72004F00754900AF3FAE3E126F008E428F4338
:103C8200C374289543FFE49542FEEF7802C333CE16
:103C920033CED8F9FFAD507C00C3EF9DF545EE9CC5
:103CA200F544C3E54464809480500675440075452C
:103CB20000E551C39450501DAF517E007C007D7FC2
:103CC200121ECA7C007D50121EDCEF2480FFEF64BE
:103CD200FFF5FA8027C3E5439428E5426480948087
:103CE2005017E550C394A050100550C3E5446480BA
:103CF200948040088545FA800375FA00AF41AE40D2
:103D0200126F008E428F43C374289543FFE495429D
:103D1200FEEF7802C333CE33CED8F9FFAD497C0033
:103D2200C3EF9DF545EE9CF544C3E5446480948061
:103D32005006754400754500E54FC39450501DAFC1
:103D42004F7E007C007D7F121ECA7C007D50121EB9
:103D5200DCEF2480FFEF64FFF5FE803BC3E5439474
:103D620028E542648094805017E549C394A050101E
:103D72000549C3E54464809480401C8545FE801754
:103D820075FE008012755100755000754F0075491F
:103D92000075FA0075FE00E508C454F0FFEF240F29
:053DA200F5468546A076
:013DA70022F9
:106E81004310000043D8000044A200004511000057
:106E91004554800045B400004622000046BD000074
:106EA10000C700C70002000A0E0F03840E0F0384FF
:106EB10000010001000000000000000000000000CF
:106DE700011400011663011200011700011A00C106
:036DF70013C19233
:030003000265ADE6
:1065AD00C0E0C083C08263A201C083C082C0D07529
:1065BD00D000C006C00720124F20134CD2B330B309
:1065CD00020512051AAF1AC3EF64809488401CAF00
:1065DD0017EF3395E0FE74402FF58274003EF5837E
:1065ED00E512F07512000517751A00E5122512F562
:1065FD0012C3E51764809484404F751700D2139031
:10660D000048E0FF8F12804120123E30133BE5120F
:10661D002512F512A2D792B3051AAF1AC3EF6480F3
:10662D009488401A0517AF17EF3395E0FE74482F85
:10663D00F58274003EF583E0FF8F12751A00C3E5F5
:10664D0017648094A04002D212D007D006D0D0D0CB
:0D665D0082D08363A201D082D083D0E032CE
:1054B100900048E56EF0A3E56FF0E56B2484FFE50D
:1054C1006A3403FE90004AEEF0A3EFF09001FBE096
:1054D100FEA3E0FF90004CEEF0A3EFF09001F9E0A5
:1054E100FEA3E0FFEF2484FFEE3403FE90004EEEB6
:1054F100F0A3EFF0E50B2484FFE50A3403FE9000EE
:1055010050EEF0A3EFF0900022E0FEA3E0FF900048
:1055110052EEF0A3EFF0900024E0FEA3E0FF900034
:1055210054EEF0A3EFF0900028E0FEA3E0FF90001E
:1055310056EEF0A3EFF0900058E54AF0A3E54BF0EA
:10554100300F0B90005AE4F0A37401F08008900032
:105551005AE4F0A3E4F0900015E0FFEF3395E0FE8C
:1055610090005CEEF0A3EFF0900014E0FFEF3395B4
:10557100E0FE90005EEEF0A3EFF0900013E0FFEF8D
:105581003395E0FE900060EEF0A3EFF0900012E0A2
:10559100FFEF3395E0FE900062EEF0A3EFF0900094
:1055A10011E0FFEF3395E0FE900064EEF0A3EFF021
:1055B100900041E0F516900040E4F0A37463F0C35D
:1055C100E5166480948840030256A2C3E516648000
:1055D100948050030256A2900042E0F518A3E0F532
:1055E10019AF16EF3395E0FEEF25E0FFEE33FE74C1
:1055F100A12FF582746E3EF583E493FE740193FF4F
:10560100D3E5199FEE6480F8E5186480984021AFD6
:1056110016EF3395E0FEEF25E0FFEE33FE74A12F88
:10562100F582746E3EF583E493F518740193F519D0
:10563100AF16EF3395E0FEEF25E0FFEE33FE74B1D8
:105641002FF582746E3EF583E493FE740193FFC3DC
:10565100E5199FEE6480F8E5186480985021AF1633
:10566100EF3395E0FEEF25E0FFEE33FE74B12FF549
:1056710082746E3EF583E493F518740193F519AFC6
:1056810016EF3395E0FEEF25E0FFEE33FE74222F97
:10569100F58274003EF583E518F0A3E519F0125187
:0C56A1003CE516B40805A20FB3920F22DE
:03002B000264E884
:1064E800C0E0C0F0C083C08263A201C083C082C084
:1064F800D075D000C000C001C002C003C004C005F0
:10650800C006C00775A61E75A6E11509AF09EF708C
:106518007030186D75090453907790003AE0FEA327
:10652800E0FFEF8EF01220AB65580000655D0001BA
:106538006562000265670003656C0004657100050B
:1065480065760006657B00076580000800006583A6
:1065580012691D8026126AF98021126CB9801C12FA
:106568005FF6801712000E8012125DCA800D125E4F
:10657800E28008126104800312585F439088123841
:10658800B2C2CFD007D006D005D004D003D002D0F5
:1065980001D000D0D0D082D08363A201D082D08332
:0565A800D0F0D0E0324C
:03002300026D4922
:106D4900C0E0C0F0C083C08263A201C083C082C01A
:106D5900D075D000C000C001C002C003C004C00586
:106D6900C006C007C2AC30981AC298E599B43F036F
:106D7900125289E599B4210B1256ADD214D215D20B
:106D890016D217C299D2ACD007D006D005D004D0FC
:106D990003D002D001D000D0D0D082D08363A20129
:096DA900D082D083D0F0D0E0329A
:03000B0002666A20
:10666A00C0E0C0F0C083C08263A201C083C082C000
:10667A00D075D000C000C001C002C003C004C0056C
:10668A00C006C007758A00758C4C75A61E75A6E1F2
:10669A00E513B42802C2960514AF14C3EF648094BC
:1066AA008A4016301213751400751700751A00C245
:1066BA0013C2127512001254B1E51375F007121EB7
:1066CA0050AFF0EF701B12422B301804D214D217BD
:1066DA00E5766007301804D215D21612002E125031
:1066EA008D1513AF13EF700C75134ED218301804B2
:1066FA00D215D216D007D006D005D004D003D002C6
:10670A00D001D000D0D0D082D08363A201D082D071
:06671A0083D0F0D0E03254
:10224500758FFF758921758DFF438780759850D2ED
:102255008CD28ED2CA75CB4C75CA0043B71143B820
:1022650021D28875D90243D84075DA4275DE42C25B
:10227500187513467509017F02125D14125D6175AB
:102285007700900040E4F0A37463F020A003126B84
:102295009375A8B275A70712514912516BC20F90D9
:1022A500006CE0FEA3E0FFEF4E6004D2108002C296
:1022B50010900068E0F560A3E0F56190006AE0F534
:1022C5005AA3E0F55BE57670FC900036E0FCA3E0F0
:1022D500FDEC121B977B007A0079207841121A7762
:1022E5007B007A00793478C312187D9001E2E0F81A
:1022F500A3E0F9A3E0FAA3E0FB12196E90001E1209
:102305002028900038E0FCA3E0FDEC121B977B0031
:102315007A0079207841121A777B007A0079B478AF
:10232500C212187D9001E2E0F8A3E0F9A3E0FAA358
:10233500E0FB12196E90001A122028900011E0FCA3
:10234500EC121B9C7B007A0079B47844121A77C092
:1023550004C005C006C007900012E0FCEC121B9CEF
:102365007B007A0079C07841121A77A804A905AADA
:1023750006AB07D007D006D005D00412187DC004DF
:10238500C005C006C007900010E0FCEC121B9C7B4A
:10239500007AC079A87847121A77A804A905AA0671
:1023A500AB07D007D006D005D00412187D900044A5
:1023B500122028900014E0FFEF3395E0FEFDFCEFBE
:1023C5002409FFEE3400FEED3400FDEC3400FC7B07
:1023D5000C7A0079007800126DFBA804A905AA06FD
:1023E500AB07900015E0FFEF3395E0FEFDFCEF2411
:1023F500D0FFEE3407FEED3400FDEC3400FCEB2F8E
:10240500FFEA3EFEE93DFDE83CFC7B077A007900EA
:102415007800121F287B047A0079007800126DFB82
:10242500C004C005C006C007900015E0FFEF339556
:10243500E0FEFDFC7B6F7A0179007800121F28D041
:1024450003D002D001D000C3EF9BFFEE9AFEED99B9
:10245500FDEC98FCC004C005C006C007900014E060
:10246500FFEF3395E0FEFDFC7B137A0179007800E0
:10247500121F287B097A0079007800126DFBA804E9
:10248500A905AA06AB07D007D006D005D004EB2FC7
:10249500FBEA3EFAE93DF9E83CF8900013E0FFEF6E
:1024A5003395E0FEFDFCEB2FFFEA3EFEE93DFDE83E
:1024B5003CFCEF247AF511EE34E0F510ED3400F52F
:1024C5000FEC3400F50E900028E0FEA3E0FFEF646A
:1024D500014E70487B017A007908C003C002C00133
:1024E5007B017A0079789001ABEBF0A3EAF0A3E9E0
:1024F500F0AF11AE10AD0FAC0E9001AE12202890CA
:102505000044E0FCA3E0FDA3E0FEA3E0FF9001B2E0
:10251500122028D001D002D003124676900028E080
:10252500FEA3E0FFEF4E60030227BF7B017A00792F
:1025350008C003C002C0017B017A007978900123AD
:10254500EBF0A3EAF0A3E9F0AF11AE10AD0FAC0EBE
:10255500900126122028900044E0FCA3E0FDA3E0B2
:10256500FEA3E0FF90012A122028D001D002D0035B
:10257500122B94AF11AE10AD0FAC0EC004C005C048
:1025850006C007900044E0FCA3E0FDA3E0FEA3E045
:10259500FF90015E122028D007D006D005D0041286
:1025A5000D47A804A905AA06AB077F007E3E7DC698
:1025B5007C481218797B007A00797A7844121A7768
:1025C500A804A905AA06AB077F007EC07D3C7C4513
:1025D500121879C004C005C006C00790001AE0FCB7
:1025E500A3E0FDA3E0FEA3E0FF125A4BA804A90552
:1025F500AA06AB07D007D006D005D00412196EC0C5
:1026050004C005C006C007900016E0FCA3E0FDA3CA
:10261500E0FEA3E0FF125A61A804A905AA06AB07CC
:10262500D007D006D005D00412196EC004C005C06D
:1026350006C007900078E0FCA3E0FDA3E0FEA3E060
:10264500FF125A4BA804A905AA06AB07D007D00666
:10265500D005D00412196EC004C005C006C007AF6E
:1026650011AE10AD0FAC0EC004C005C006C0077F8B
:10267500AB7EAA7D0A7CBF900044E0F8A3E0F9A3F5
:10268500E0FAA3E0FB12187D90015E122028D00726
:10269500D006D005D004120D47C004C005C006C041
:1026A50007AF11AE10AD0FAC0EC004C005C006C01B
:1026B500077F007E007D207CBF900044E0F8A3E00A
:1026C500F9A3E0FAA3E0FB12187D90015E12202821
:1026D500D007D006D005D004120D47D003D002D0C4
:1026E50001D0001218797B337A337993783F121A27
:1026F50077A804A905AA06AB07D007D006D005D050
:102705000412187D121BD08E0C8F0D90003CE0FE3C
:10271500A3E0FFC3EF9404EE64809480504FAC0CAB
:10272500AD0DEC121B97C004C005C006C007900094
:102735003CE0FEA3E0FFEF7802C333CE33CED8F9F9
:10274500FF74812FF582746E3EF583121FF8D00752
:10275500D006D005D00412196E7B007A00797A78FC
:1027650044121A77121BD08E1B8F1C804DAC0CADFA
:102775000DEC121B97C004C005C006C00790003CB5
:10278500E0FEA3E0FFEF7802C333CE33CED8F9FFE6
:1027950074812FF582746E3EF583121FF8D007D031
:1027A50006D005D00412196E7B007A40791C784654
:1027B500121A77121BD08E1B8F1C900028E0FEA3E7
:1027C500E0FFEF64024E70149000781220343F82CF
:1027D500D0E590000812203440C39DB2900028E057
:1027E500FEA3E0FFEF64034E7014900078122034CE
:1027F5003F3566CF90000812203440A73B64900017
:1028050028E0FEA3E0FFEF64044E701490007812F8
:102815002034BF018FC590000812203440953F7DBC
:10282500900028E0FEA3E0FFEF64054E70149000D1
:10283500781220343EC44D019000081220343FB96F
:102845001687900028E0FEA3E0FFEF64064E7014A3
:102855009000781220343F32B6AE90000812203432
:10286500401F2B02900028E0FEA3E0FFEF64074E17
:1028750070149000781220340000000090000812B7
:10288500203440BC7AE1900028E0FEA3E0FFEF642D
:10289500084E7067900032E0FCA3E0FDEC121B9738
:1028A5007B007A0079207841121A779001E2E0F8EE
:1028B500A3E0F9A3E0FAA3E0FB12196E9000081259
:1028C5002028900034E0FCA3E0FDEC121B977B0070
:1028D5007A0079207841121A777B007A0079B478EA
:1028E500C212187D9001E2E0F8A3E0F9A3E0FAA393
:1028F500E0FB12196E900078122028900028E0FE67
:10290500A3E0FFC3EF9409EE648094804003022A9C
:1029150013900044E0FCA3E0FDA3E0FEA3E0FFC0AC
:1029250004C005C006C007AF11AE10AD0FAC0E90C8
:1029350001CE122028D007D006D005D004124A3E79
:102945009001881220287B017A00790CC003C0020F
:10295500C0017B017A007900900185EBF0A3EAF0D4
:10296500A3E9F0900008E0FCA3E0FDA3E0FEA3E0EE
:10297500FF90018C122028900078E0FCA3E0FDA3D5
:10298500E0FEA3E0FF900190122028D001D002D0F4
:102995000312339B900028E0FEA3E0FFEF4E705A30
:1029A500900000E0FCA3E0FDA3E0FEA3E0FF125AC7
:1029B5004B7B007A5079C7784512196EC004C00563
:1029C500C006C0079000E812203448B98C00D00733
:1029D500D006D005D004126A5CA804A905AA06ABE6
:1029E50007900000E0FCA3E0FDA3E0FEA3E0FF12DA
:1029F50018799000041220288014900000E0FCA3B0
:102A0500E0FDA3E0FEA3E0FF900004122028900063
:102A150028E0FEA3E0FFEF64094E705C90002EE015
:102A2500FCA3E0FDEC121B977B007A00792078412E
:102A3500121A779001E2E0F8A3E0F9A3E0FAA3E027
:102A4500FB12196E90000C122028900030E0FCA3B8
:102A5500E0FDEC121B977B007A0079207841121A71
:102A6500779001E2E0F8A3E0F9A3E0FAA3E0FB1216
:102A7500196E900004122028900028E0FEA3E0FFC4
:102A8500EF640A4E705C90002AE0FCA3E0FDEC12B6
:102A95001B977B007A0079207841121A779001E222
:102AA500E0F8A3E0F9A3E0FAA3E0FB12196E9000A9
:102AB5000C12202890002CE0FCA3E0FDEC121B97E3
:102AC5007B007A0079207841121A779001E2E0F8CC
:102AD500A3E0F9A3E0FAA3E0FB12196E900004123B
:102AE50020289001E2E0F8A3E0F9A3E0FAA3E0FBD7
:102AF50090000CE0FCA3E0FDA3E0FEA3E0FF121AAA
:102B0500777BCD7ACC794C783D12187D7B007A00A5
:102B15007920784112196E121BD08E6E8F6F90013D
:102B2500E2E0F8A3E0F9A3E0FAA3E0FB900004E0FB
:102B3500FCA3E0FDA3E0FEA3E0FF121A777BCD7AAC
:102B4500CC794C783D12187D7B007A00792078414C
:102B550012196E121BD08E6A8F6B7F007E007D204E
:102B65007C41900078E0F8A3E0F9A3E0FAA3E0FB4C
:102B750012196E9001E2E0F8A3E0F9A3E0FAA3E0F0
:0F2B8500FB121A77121BD08E0A8F0B0222CA2264
:105CAD00EFC0E0C283740F125CE27430125CEC74CE
:105CBD0005125CE27430125CEC7401125CE274301B
:105CCD00125CEC7401125CE2D0E0146002740844C2
:105CDD0020125CFA227D000000DDFCD5E0F7225495
:105CED00F053800F4280C282D283C28322C282804F
:105CFD0002D282C0E0125D08D0E0C454F053800F90
:105D0D004280D283C28322125CAD125D46740612AC
:105D1D005CFA125D46740E125CFA125D4674011245
:105D2D005CFA125D467440125CFA125D93125D4688
:105D3D007480125CFA125D7322740A125CE222EF17
:105D4D00C0E0125D46D0E0125CFE22125D46740288
:105D5D00125CFA22125D467401125CFA22125D4643
:105D6D00740E125CFA22125D46740C125CFA221249
:105D7D005D46740F125CFA22EFC0E0125D46D0E072
:105D8D004480125CFA22905DA27E28E493FF125D9E
:105D9D004CA3DEF7220004040E0E1F1F00001F1F70
:105DAD000E0E04040000101C1F1C10000000010743
:0D5DBD001F070100000E11171917110E002D
:106EE8007A107B00EE6BFB8BF053F080ABF033EF46
:086EF80033FFEE33FEDAEE2257
:106C2800900207EEF0A3EFF0900207E0FEA3E0FF6A
:106C38007C037DE8121EDCEF2430F5993099FDC203
:106C480099900207E0FEA3E0FF7C037DE8121EDCBA
:106C58007E007F64CFCDCFCECCCE121EDCEF2430A9
:106C6800F5993099FDC299900207E0FEA3E0FF7CF8
:106C7800007D64121EDC7E007F0ACFCDCFCECCCE45
:106C8800121EDCEF2430F5993099FDC29990020765
:106C9800E0FEA3E0FF7C007D0A121EDCAF05EF24B6
:106CA80030F5993099FDC2997599003099FDC299CE
:016CB80022B9
:105289009001FD122034000186A020983E9001FD76
:10529900E0FCA3E0FDA3E0FEA3E0FFEC4D4E4F6070
:1052A9002A9001FDE0FCA3E0FDA3E0FEA3E0FF7B63
:1052B900FF7AFF79FF78FFEF2BFFEE3AFEED39FD1C
:1052C900EC38FC9001FD12202880BFC298AF99EFFD
:1052D900122085532E61533A62534663534E6453E9
:1052E9005A65536666537267537E68538A69539643
:1052F9006A53A26B53AE6C53BA6D53C66E53D46FD7
:1053090053E07053F47153FC72540A735418745473
:105319005D75546B7654797754877854957954A38D
:105329007A000054B0900022E0FEA3E0FF126C283E
:1053390022900024E0FEA3E0FF126C2822AF4BAEBE
:105349004A126C2822900028E0FEA3E0FF126C2884
:105359002290002AE0FEA3E0FF126C282290002C84
:10536900E0FEA3E0FF126C282290002EE0FEA3E0ED
:10537900FF126C2822900030E0FEA3E0FF126C2897
:1053890022900032E0FEA3E0FF126C282290003444
:10539900E0FEA3E0FF126C2822900036E0FEA3E0B5
:1053A900FF126C2822900038E0FEA3E0FF126C285F
:1053B9002290003AE0FEA3E0FF126C2822E50D24BA
:1053C90088FFE50C3413FE126C28229001FBE0FEE5
:1053D900A3E0FF126C28229001F9E0FEA3E0FFEFA1
:1053E9002484FFEE3403FE126C2822AF6FAE6E12D6
:1053F9006C2822E56B2484FFE56A3403FE126C28CD
:1054090022E50B2484FFE50A3403FE126C2822A24C
:105419000FE433FFEF3395E0FEEFC4F8540FC8688B
:10542900FFEEC454F048FEE5A0C4540FFD7C00EF24
:105439002DFDEE3CFCA210E433FFEF3395E0FEEFC7
:105449007805C333CE33CED8F9FFED2FFFEC3EFEFE
:10545900126C2822900010E0FFEF3395E0FE126CE9
:105469002822900011E0FFEF3395E0FE126C28220C
:10547900900012E0FFEF3395E0FE126C28229000B5
:1054890013E0FFEF3395E0FE126C2822900014E040
:10549900FFEF3395E0FE126C2822900015E0FFEF34
:0754A9003395E0FE126C28B0
:0154B00022D9
:106878009001EEE4F0A3E4F09001F4E4F09001F468
:10688800E0FFD3EF6480948340030269149001F021
:10689800122034000186A020983E9001F0E0FCA36D
:1068A800E0FDA3E0FEA3E0FFEC4D4E4F602A90010F
:1068B800F0E0FCA3E0FDA3E0FEA3E0FF7BFF7AFF8E
:1068C80079FF78FFEF2BFFEE3AFEED39FDEC38FC4F
:1068D8009001F012202880BFC2989001EEE0FEA33C
:1068E800E0FF7C007D0A121ECAAD997C00EF2DFFE7
:1068F800EE3CFEEF24D0FFEE34FFFE9001EEEEF00A
:10690800A3EFF09001F4E004F00268859001EEE056
:04691800FEA3E0FFFB
:01691C002258
:1056AD00900201122034000186A020983E90020144
:1056BD00E0FCA3E0FDA3E0FEA3E0FFEC4D4E4F6048
:1056CD002A900201E0FCA3E0FDA3E0FEA3E0FF7B36
:1056DD00FF7AFF79FF78FFEF2BFFEE3AFEED39FDF4
:1056ED00EC38FC90020112202880BFC298AF99EFD0
:1056FD001220855746615755625764635773645737
:10570D00826557916657A06757AF6857BE6957CDE9
:10571D006A57DC6B57EB6C57FA6D580972580E735C
:10572D00581174581775582376582F77583B785859
:10573D00477958537A0000585E126878900022EE2F
:10574D00F0A3EFF012513C22126878900024EEF095
:10575D00A3EFF012513C22126878900026EEF0A3D0
:10576D00EFF012513C22126878900028EEF0A3EF72
:10577D00F012513C2212687890002AEEF0A3EFF05F
:10578D0012513C2212687890002CEEF0A3EFF0122B
:10579D00513C2212687890002EEEF0A3EFF01251DA
:1057AD003C22126878900030EEF0A3EFF012513CDD
:1057BD0022126878900032EEF0A3EFF012513C22E5
:1057CD00126878900034EEF0A3EFF012513C2212E3
:1057DD006878900036EEF0A3EFF012513C2212687B
:1057ED0078900038EEF0A3EFF012513C2212687859
:1057FD0090003AEEF0A3EFF012513C22D20DD211EF
:10580D0022D21122A20FB3920F22126878900010AB
:10581D00EFF012503822126878900011EFF012500C
:10582D003822126878900012EFF012503822126868
:10583D0078900013EFF0125038221268789000140F
:10584D00EFF012503822126878900015EFF01250D8
:01585D003812
:01585E002227
:10187600021C3CE86480F8E933E83360110460F048
:10188600ED33EC337009E8FCE9FDEAFEEBFF2204D8
:1018960060DED3EB9FEA9EE99DE8C2E78CF0C2F7D3
:1018A60095F0400CE8CCF8E9CDF9EACEFAEBCFFB9F
:1018B600121C0785D0F05804700320D5B3E80470D5
:1018C600075002B2D5021C4692D5EC0460F7E4CC70
:1018D600C0E0C398F8603B94186008400DD0E0FB68
:1018E600021C1EE4FBFAC9FC8028E830E406E4C9C1
:1018F600FBE4CAFCE830E305E4C9CACBFCE85407BC
:101906006010F8C3E913F9EA13FAEB13FBEC13FCC6
:10191600D8F130F52FC3E49CFCEF9BFFEE9AFEED69
:1019260099FDD0E0FBEF4E4D4C701222DB03021CFA
:1019360043EC2CFCEF33FFEE33FEED33FDED30E7E9
:10194600EB021C1EEF2BFFEE3AFEED39FDD0E0FB5D
:1019560050130BBB0003021C46ED13FDEE13FEEF06
:0819660013FFEC13FC021C1E30
:10196E00EC4D6011E8497017ED33EC3304600DE473
:10197E00FCFFFEFD22E933E8330470F8021C3C1232
:10198E001C0758046009E4CC248150062850090233
:10199E001C46284003021C43C0E0EB4A7044B98049
:1019AE0006D0E0FB021C32EF4E701CBD8008EBFF30
:1019BE00EAFEE9FD80EBE98DF0A4FEE5F0021A5790
:1019CE00E9CDF9EAFEEBFFEF89F0A4FCE5F0CE8954
:1019DE00F0A42EFFE435F0CD89F0A42DFEE435F011
:1019EE008067EF4E7005BD80D780C3EF8BF0A4AC3F
:1019FE00F0EE8BF0A42CFCE435F0F8EF8AF0A42C7A
:101A0E00E5F038FCE433CB8DF0A42CFCE5F03BF88C
:101A1E00EE8AF0A42CFCE5F038F8E433CF89F0A47C
:101A2E002CFCE5F038CF3400CE89F0A42FFFE5F082
:101A3E003EFEE433C98DF0A42EFEE5F039CD8AF0DA
:101A4E00A42FFFE5F03EFEE43DFD33D0E0FB500752
:101A5E000BBB000F021C46EC2CFCEF33FFEE33FEEB
:061A6E00ED33FD021C1E19
:101A7400021C46EC5D046005E859047003021C3C3A
:101A8400121C07580460F6EC4860F2EC7004FDFE8A
:101A9400FF22C860DB2481C85009C3986002500645
:101AA400021C439850CAF582E9294B4A7005AB825F
:101AB400021C3275F0007C1A7880C3EF9BEE9AED1D
:101AC40099400DC3EF9BFFEE9AFEED99FDE842F0BD
:101AD400DC23ACF0D0E0FFD0E0FED0E0FDAB822010
:101AE400E7101BEB60BAEC2CFCEF33FFEE33FEED9A
:101AF40033FD021C1EE803F830E705C0F075F00062
:101B0400EF2FFFEE33FEED33FD40B830E7C280AA7D
:101B140074F8CC6480CCC86480C8F582046043C384
:101B2400EB9FF5F0EA9E42F0E99D42F0E89C45F017
:101B340060305018E5825FFFE582F42B5582FB503C
:101B4400210ABA001D09B90019088016E5825BFB59
:101B5400E582F42F5582FF50090EBE00050DBD002D
:101B6400010CC3EB9FF5F0EA9E42F0E99D42F0E8D8
:0D1B74009C45F06007CC4820E701B3EC224F
:101B8100ED33EC33600A047003BD8004ECB2E7FC72
:011B91002231
:101B920075F020800E75F010800575F0087D007ECE
:101BA200007F003392D530D503121F77EC334010FB
:101BB200EF33FFEE33FEED33FDEC33FCD5F0ED22D7
:0E1BC200E5F0247EA2D513CC92E7CDCEFF2213
:101BD000EDD2E7CD33EC3392D524814006E4FFFE0D
:101BE000FDFC22FCE4CFCECDCC24E0501174FF806C
:101BF000EDC3CC13CCCD13CDCE13CECF13CF047009
:071C0000F030D5DE021F7772
:103DA800E57B24F3F582E43400F583E0057B22907B
:103DB80000F03009039000F3E475F0011220650269
:103DC8001E722002E97F2ED2028018EF540F249031
:103DD800D43440D4FF30060BEF24BFB41A0050038C
:103DE8002461FFE57C6002157C057FE57F70020594
:103DF8007E30090E9000F0E475F001122065EF02A4
:103E08001EB8026EC17403D2098003E4C209F57BAF
:103E18009000F012207CE4F57CF57EF57FE57C606F
:103E2800077F20123DEB80F5757DFFC203C202C2F9
:103E380004C205C207C208C20A123DB7FF700D309E
:103E480009057F00123DFCAF7FAE7E22B4255FC21C
:103E5800D5C206123DB7FF24D0B40A00501A75F037
:103E68000A787C30D50508B6FF0106C6A426F620D8
:103E7800D5047002D20580D924CFB41A00EF5004BB
:103E8800C2E5D2060240EED20380C6D20280C0D27A
:103E98000480BCD2D580BAD20780B47F20123DEB13
:103EA8002004077401B57C0040F1123DA8FF123DC3
:103EB800EB023E25D20AD2088095123DA8FB123D9E
:103EC800A8FA123DA8F94A4B700679EC7A417BFFB3
:103ED80020042EE57C602A7E008E82758300121EE7
:103EE8008B60060EEE657D70F0C2D5EBC0E0EAC0CF
:103EF800E0E9C0E0EE12414FD0E0F9D0E0FAD0E0BE
:103F0800FB121E72FF60AAEBC0E0EAC0E0E9C0E065
:103F1800123DEBD0E02401F9D0E03400FAD0E0FB08
:103F2800E57D0460DCD57DD98087D20480A212416A
:103F38003160F7E57D700104121C51A97D600DE523
:103F48007D600914F57D1241D9EF60F3EA30E7028C
:103F5800F404C3995079EAF4257D0430E701E404B8
:103F6800F57D800D12413160C1EA057D257D121C69
:103F780051EA90011FF030E701E4257D04D57D0466
:103F88002007011412414FE4C0E01241D990011FEB
:103F9800E0601320E70714F0123DD3802204F0D02C
:103FA800E014C0E07F00123DD3E57D6007123DCAF2
:103FB800157D800B300703123DCAD0E0023E25D0A4
:103FC800E00480C4124131609EE57D04121C5190CA
:103FD800011FEAF0E57D2007026001042404124174
:013FE8004F89
:103FE90074FF04C0E01241D9123DD3E57D200702D8
:103FF9006003123DCAD0E0B57DE87F45123DDD90F2
:10400900011FE07F2B30E7047F2DF404C0E0123D4F
:10401900EBD0E075F00A84C0F0123DD4D0E0123D37
:10402900D4023E25791080027908C208C20A8008A4
:10403900D2D5790A8004790AC2D5E57D047002F5E2
:104049007DE4FAFDFEFF123DA8FC7B082003131254
:104059003DA8FD7B1030020A123DA8FE123DA8FFC3
:104069007B20EC3382D592D55013C3E43002069FEE
:10407900FFE49EFEE42003039DFDE49CFCE4CBF8F1
:10408900C203EC700CCFCECDCCE824F8F870F380E5
:1040990017C3EF33FFEE33FEED33FDEC33FCEB33A7
:1040A900FB994002FB0FD8E9EB300305F8D0E0C4D7
:1040B90048B203C0E00AEC4D4E4F78207B0070C235
:1040C900EAB57D0040BCC0E0124151D0F0D0E020FB
:1040D9000304C4C0E0C4B203C0F0123DD4D0F0D58B
:1040E900F0EB023E251220853EC253402D583E93E7
:1040F9004C3E8F4240314F4039444039493EA843F4
:10410900403F553F6C463FCC453F3647420C503EF9
:10411900972D3E9B2E3EBE2B3E9F233EBC2041F554
:104129002A3E574800003EB6E57DB4FF03757D067B
:10413900123DA8FC123DA8FD123DA8FE123DA8FFA4
:10414900900118021C8E790AA2D52005143007099E
:10415900B910020404B9080104A2D52008025001CB
:10416900042004689204B57C005034C0E07F2030FC
:1041790005197F30A20472087207500F1241A8C2B4
:1041890004C208C207C20A7F30800F300703E9C0A2
:10419900E0123DEB300703D0E0F9D0E0B57CCC303C
:1041A90007177F30B9100C123DEB7F583006077F97
:1041B900788003B90803123DEB3004057F2D023DD9
:1041C900EB7F20200AF87F2B2008F322920480CF6E
:1041D9007F00B40700500B2418F582E43401F583FD
:1041E900E0FF22286E756C6C2900D203123DA830BD
:1041F90003F8C203787C30D50108F6023E572D50EA
:10420900434958123DA82403B405004001E49042F3
:104219000793123DDC743A123DDCD205757C040229
:02422900402D26
:0D6F7800ED33EC3360065004EC6480FC2225
:1067CC00021C3C22EDA2E7D2E7F9EC3340F260F375
:1067DC00B4FF08ED547F70E8021C46F82481C2E037
:1067EC00C0E0F40428FAC313FCED92E7FD9000E43A
:1067FC00122028EEA2E7E9BA7F02C31334009400FA
:10680C00FA75F091A4E5F013F494FE8AF0A433E544
:10681C00F033248CD313FDE492E7FE7F007C3F75AC
:10682C008302ECC0E0F8EDC0E0F9EEC0E0FAEFC096
:10683C00E0FB8583F09000E4121FD085F083121AE0
:10684C0077D0E0FBD0E0FAD0E0F9D0E0F812187D78
:10685C00ED6480FD30E7011CD583C7ED33CC33F8F4
:0C686C00D0E0A2E71328C313CC13FD22D8
:106A5C009000E41220289000E8E0F8A3E0F9A3E00D
:106A6C00FAA3E0FB9000E4E0FCA3E0FDA3E0FEA3AE
:106A7C00E0FF121A77125BAB9000E4122028900012
:106A8C00E8E030E7599000E4E0FCA3E0FDA3E0FE71
:106A9C00A3E0FFECC0E0EDC0E0EEC0E0EFC0E0E44E
:106AAC00FFFEFDFC9000E4E0F8A3E0F9A3E0FAA3FC
:106ABC00E0FB121B147BDB600250087A0F794978DB
:106ACC004080067A0F794978C0D0E0FFD0E0FED044
:106ADC00E0FDD0E0FC12187D9000E412202890001C
:0D6AEC00E4E0FCA3E0FDA3E0FEA3E0FF2238
:105A03003A70FA83BCAAE9E43E81E0F8BF9DE9E677
:105A13003F80000039283C1ABB9969663DA335E3F2
:105A2300BF255DE73FC90FDB418DDBCCC44936EEB3
:105A330045C9913FC5B0F83D3F800000C317F53419
:105A4300452FFA73C60AFDDD125B0C04A2E1920036
:105A53001420E015905A037404121D938030125BD6
:105A63000C30E102B20020E0EBA883A9829000E4AD
:105A730012202889828883905A177404121D9385F3
:105A830082F09000E4121FEC85F08212196EED4C47
:105A93006007300004EC6480FC22125B0CC0E0A8B9
:105AA30083A9829000E412202889828883905A3B3C
:105AB3007403121D938582F09000E4121FEC85F0AD
:105AC3008212196E9000E4E0CCF0A3E0CDF0A3E0E5
:105AD300CEF0A3E0CFF0905A2B7403121D93D08223
:105AE3008582F09000E4121FEC85F082E58230E0BD
:105AF30007121A77B2008096EFCBFFEECAFEEDC90C
:105B0300FDECC8FC121A778085ED33EC547FCC335F
:105B1300920024605007D0E0D0E0021C3C7B837AE3
:105B2300F97922783E12196EEDF933ECF8332481BA
:105B33005011EFFBEEFA121BD0121B92ECB2E7FCF2
:105B430012187DED33EC33602F2403F8C313FCEDFF
:105B530092E7FDE82481E4501FECF8EDF9EEFAEF4B
:105B6300FB121BD0EF04C2E0FCF582121B9CECB2CB
:105B7300E7FC12187DE58203FAED33EC336007147A
:085B830013FCED92E7FDEA229C
:105B8B00BE1249253E4CCCCDBEAAAAAB3F8000002D
:105B9B003E7ADBB03EED63383F24BC7D3F490FDBE3
:105BAB00ED33ECC2E7CC339200B4FF13ED547F60BE
:105BBB0003021C3C7FDB7E0F7DC97C3F025CA0C2D5
:105BCB0001C3947F401E7007EDD2E794904015EF10
:105BDB00FBEEFAEDF9ECF87F007E007D807C3F1246
:105BEB001A77D201ED33EC33248430E705E4C0E0BF
:105BFB00806B04FAEDD2E754F0C333DAFD5407346B
:105C0B00002323C0E0CCC0E0F8EDC0E0F9EEC0E02B
:105C1B00FAEFC0E0FBE4121B9CEC24FEFC9000ECC2
:105C2B0012202812196E7B007A007980783F1218A7
:105C3B007D9000ECE0B2E7CCF0A3E0CDF0A3E0CE9A
:105C4B00F0A3E0CFF0D0E0FBD0E0FAD0E0F9D0E069
:105C5B00F812187D9000EC121FEC121A779000ECE2
:105C6B00122028905B8B7403121D939000EC121F73
:105C7B00EC12196ED0E0600F2497F582E4345BF5DB
:105C8B0083121FF812187D30010B7BDB7A0F79C959
:105C9B0078BF12187DED33EC336006ECA20092E76F
:025CAB00FC22D9
:106311009000E412202874FFFFFEFDFC9000E4E0F1
:10632100F8A3E0F9A3E0FAA3E0FBC3121F856038EC
:106331007F807E967D187C4B9000E4E0F8A3E0F925
:10634100A3E0FAA3E0FB121B146002501B7F807EC6
:10635100967D187CCB9000E4E0F8A3E0F9A3E0FA85
:10636100A3E0FB121B14500F9000E4E0FCA3E0FD3E
:10637100A3E0FEA3E0FF229000E4E0FCA3E0FDA384
:10638100E0FEA3E0FF121BD09000E812202890004D
:10639100E8E0FCA3E0FDA3E0FEA3E0FFEC121B920A
:1063A100C8ECC8C9EDC9CAEECACBEFCB9000E4E096
:1063B100FCA3E0FDA3E0FEA3E0FF121879E4FBFAE1
:1063C100F9F8121B14602640249000E8E0FCA3E0D9
:1063D100FDA3E0FEA3E0FFEF24FFFFEE34FFFEED9F
:1063E10034FFFDEC34FFFC9000E81220289000E817
:1063F100E0FCA3E0FDA3E0FEA3E0FFEC121B922270
:101C0700E9D2E7C933E833F892D5EDD2E7CD33EC23
:071C170033FC5002B2D5229C
:101C1E00EC30E7100FBF000C0EBE00080DBD000427
:101C2E000BEB6014A2D5EB13FCED92E7FD2274FFD3
:101C3E00FCFDFEFF22E480F8A2D574FF13FC7D802C
:031C4E00E480EF40
:101C5100F920E73624F950037907E4F42402FBE57F
:101C610082158270021583DBF6E024FB501BE960CC
:101C710014E4F0E582158270021583E004F0B40AE1
:0D1C810008E4F0D9EE7401F00A22C2D52269
:101C8E00ED33EC3392D5FA602AB4FF33EDC2E77B25
:101C9E00FF60067A1C79B3E4227A1C79BC20D50445
:101CAE007A1C79B7224E614E002B494E46002D49C3
:101CBE004E4600E47A08F0A3DAFC7B00740722C0DB
:101CCE0083C082ECC0E0EDC0E0EEC0E0EFC0E0EA21
:101CDE0075F010A4CAABF075F04DA42BFBE435F0F3
:101CEE00FCEA2410FAEB34C5FBEC34D9FCEDC2E768
:101CFE00FF75F056A4F42411C5F0F434C58FF0A48A
:101D0E002AE5F03BE43CF020E714121E10D0E0FF71
:101D1E00D0E0FED0E0FDD0E0FC121A778014F4047F
:101D2E00121E10D0E0FFD0E0FED0E0FDD0E0FC129D
:101D3E00196ED082D083E0FAEDD2E7CD33EC3324A6
:101D4E0082FBE4C3CF33CFCE33CECD33CD33DBF3F3
:101D5E007B0775F00A846004F0A31B0AE5F0F0A37C
:101D6E008FF0740AA4FFACF08EF0740AA42CFEACB3
:101D7E00F050010C8DF0740AA42CFDE435F0F0A3A4
:051D8E00DBDE740722FA
:101D9300C0E0EFFBEEFAEDF9ECF812196ED0E0F5C6
:101DA300F0EFFBEEFAEDF9ECF8121FDCA3A3A3A30B
:101DB300E8C0E0E9C0E0EAC0E0EBC0E0C0F012191F
:101DC3006E121FF8A3A3A3A312187DD0F0D0E0FBDB
:0D1DD300D0E0FAD0E0F9D0E0F8D5F0D4224D
:101DE0003F8000004120000042C80000447A00000B
:101DF000461C400047C35000497424004B1896808D
:101E00004CBEBC205A0E1BCA6753C21C749DC5AE83
:101E1000FB60065407601C2323121E3EEB543860FF
:101E200009121E2A121E3912196EECF8EDF9EEFA9B
:101E3000EFCB22EB121E3980F1543803241C901D85
:101E4000E0FE93FC0EEE93FD0EEE930ECE93FF227A
:1069DC00022245E493A3F8E493A34003F68001F26A
:1069EC0008DFF48029E493A3F85407240CC8C333BC
:1069FC00C4540F4420C8834004F456800146F6DF8B
:106A0C00E4800B0102040810204080906DB2E47EFB
:106A1C00019360BCA3FF543F30E509541FFEE4937F
:106A2C00A360010ECF54C025E060A840B8E493A346
:106A3C00FAE493A3F8E493A3C8C582C8CAC583CA71
:106A4C00F0A3C8C582C8CAC583CADFE9DEE780BE29
:016DFA000098
:101E5000C2D530F707B2D563F0FF05F030E70CB21A
:101E6000D5F4048463F0FF05F080018430D502F4DA
:021E700004224A
:101E7200BB010689828A83E0225002E722BBFE026E
:091E8200E32289828A83E49322A1
:101E8B00BB010CE58229F582E5833AF583E022500C
:101E9B0006E92582F8E622BBFE06E92582F8E22256
:0D1EAB00E58229F582E5833AF583E4932270
:101EB800BB010689828A83F0225002F722BBFE0109
:021EC800F32203
:101ECA00EF8DF0A4A8F0CF8CF0A428CE8DF0A42E2C
:021EDA00FE22E6
:101EDC00C2D5EC30E709B2D5E4C39DFDE49CFCEE21
:101EEC0030E715B2D5E4C39FFFE49EFE1220D8C3A1
:101EFC00E49DFDE49CFC80031220D830D507C3E49C
:061F0C009FFFE49EFE228F
:101F1200C5F0F8A3E028F0C5F0F8E582158270025A
:061F22001583E038F022F7
:101F2800E88FF0A4CC8BF0A42CFCE98EF0A42CFC58
:101F38008AF0EDA42CFCEA8EF0A4CDA8F08BF0A4D6
:101F48002DCC3825F0FDE98FF0A42CCD35F0FCEB35
:101F58008EF0A4FEA9F0EB8FF0A4CFC5F02ECD39FA
:0F1F6800FEE43CFCEAA42DCE35F0FDE43CFC2267
:106DFB00C2D5E830E70FB2D5E4C39BFBE49AFAE4C3
:106E0B0099F9E498F8EC30E717B2D5126E311221EC
:106E1B0069E4C39BFBE49AFAE499F9E498F88003DC
:106E2B0012216930D50DE4C39FFFE49EFEE49DFD66
:046E3B00E49CFC22B5
:0E1F7700C3E49FFFE49EFEE49DFDE49CFC227B
:101F8500EB9FF5F0EA9E42F0E99D42F0E89C45F0B2
:011F95002229
:101F9600BB010789828A83021FD05005E9F8022116
:101FA600FBBBFE05E9F802220789828A83021FDC51
:101FB600BB010789828A830220285005E9F802229C
:0A1FC6002DBBFE05E9F802223922C6
:0C1FD000E0FCA3E0FDA3E0FEA3E0FF2284
:101FDC00E493FC740193FD740293FE740393FF224B
:0C1FEC00E0F8A3E0F9A3E0FAA3E0FB2278
:101FF800E493F8740193F9740293FA740393FB223F
:10200800BB010789828A83021FEC5005E9F8022286
:1020180013BBFE05E9F802222089828A83021FF891
:0C202800ECF0A3EDF0A3EEF0A3EFF0222B
:10203400A8828583F0D083D08212204B12204B12C9
:10204400204B12204BE473E493A3C583C5F0C583EE
:10205400C8C582C8F0A3C583C5F0C583C8C582C8F6
:012064002259
:10206500F8E0FBA3A3E0F925F0F0E5821582700204
:072075001583E0FA38F022A8
:09207C00EBF0A3EAF0A3E9F02265
:10208500D083D082F8E4937012740193700DA3A3EA
:1020950093F8740193F5828883E4737402936860FE
:0620A500EFA3A3A380DFFE
:1020AB00D083D082F8E4937012740193700DA3A3C4
:1020BB0093F8740193F5828883E473740293B5F0FB
:0D20CB00067403936860E9A3A3A3A380D863
:106EC100EFB40A07740D126ECC740A309811A899A8
:106ED100B8130CC2983098FDA899C298B811F63031
:076EE10099FDC299F5992209
:106F0000C3EE6480948040028007C3E49FFFE49E48
:026F1000FE225F
:1020D800BC000BBE0029EF8DF084FFADF022E4CCEC
:1020E800F875F008EF2FFFEE33FEEC33FCEE9DECB5
:1020F800984005FCEE9DFE0FD5F0E9E4CEFD22EDFB
:10210800F8F5F0EE8420D21CFEADF075F008EF2F44
:10211800FFED33FD4007985006D5F0F222C398FD35
:052128000FD5F0EA22D2
:10212D0075F008758200EF2FFFEE33FECD33CDCC69
:10213D0033CCC58233C5829BED9AEC99E5829840EC
:10214D000CF582EE9BFEED9AFDEC99FC0FD5F0D6C9
:10215D00E4CEFBE4CDFAE4CCF9A88222B800C1B9F3
:10216D000059BA002DEC8BF084CFCECDFCE5F0CB31
:10217D00F97818EF2FFFEE33FEED33FDEC33FCEB6A
:10218D0033FB10D703994004EB99FB0FD8E5E4F925
:10219D00FA227818EF2FFFEE33FEED33FDEC33FC12
:1021AD00C933C910D7059BE99A4007EC9BFCE99A06
:1021BD00F90FD8E0E4C9FAE4CCFB2275F010EF2F4B
:1021CD00FFEE33FEED33FDCC33CCC833C810D7074B
:1021DD009BEC9AE899400AED9BFDEC9AFCE899F886
:0E21ED000FD5F0DAE4CDFBE4CCFAE4C8F92219
:0C21FB00E6FC08E6FD08E6FE08E6FF2210
:0C220700E2FC08E2FD08E2FE08E2FF2213
:0D221300E6FB08E6F908E6FA08E6CBF8223B
:0D222000E2FB08E2F908E2FA08E2CBF8223E
:0C222D00ECF608EDF608EEF608EFF622DD
:0C223900ECF208EDF208EEF208EFF222E1
:00000001FF
